:020000041000EA
:1000000000B5324B212058609868022188439860DF
:10001000D860186158612E4B002199600221596106
:100020000121F02299502B49196001219960352056
:1000300000F044F80222904214D00621196600F024
:1000400034F8196E01211966002018661A6600F04E
:100050002CF8196E196E196E052000F02FF8012189
:100060000842F9D1002199601B49196000215960AB
:100070001A491B48016001219960EB211966A021F2
:10008000196600F012F800219960164914480160C1
:100090000121996001BC002800D000471248134993
:1000A000086003C880F30888084703B5996A0420EC
:1000B0000142FBD001200142F8D103BD02B5186610
:1000C0001866FFF7F2FF186E186E02BD00000240BE
:1000D000000000180000070000035F00212200005C
:1000E000F4000018222000A00001001008ED00E03C
:1000F00000000000000000000000000074B24E7A12
:1001000000200420F7010010C3010010C5010010F9
:10011000C1010010C1010010C1010010C101001097
:10012000C1010010C1010010C1010010C701001081
:10013000C1010010C1010010C9010010CB01001065
:10014000CD010010CD010010CD010010CD01001037
:10015000CD010010CD010010CD010010CD01001027
:10016000CD010010CD010010CD010010CD01001017
:10017000CD010010CD010010CD010010CD01001007
:10018000CD010010CD010010CD010010CD010010F7
:10019000CD010010CD010010CD010010CD010010E7
:1001A000CD010010CD010010CD010010CD010010D7
:1001B000CD010010CD010010CD010010CD010010C7
:1001C00000BE00BE00BE00BE00BE00BE00F04BF888
:1001D000103800BEF2EB88710CAD001030AD00108D
:1001E0003402001090A31AE700202149086006C8D5
:1001F00081F3088810471F48006800282FD10DA4FC
:100200000ECC002902D000F012F8F9E71A491B4A77
:10021000002000E001C19142FCD1194988471949E9
:1002200088471949884700BEFDE701C901C29A42C3
:10023000FBD3704730AD0010C000002048050020FF
:10024000B8B100100000042000000420B8B1001074
:1002500000100420001004200000000070470B482C
:1002600005F078F80047EFF30580C0B27047000052
:1002700008ED00E0000000D000800020B08E0220D9
:10028000813C00109D1E00103D3C001057560000A0
:1002900006005250ABB3605374A3001006005250D6
:1002A000861C030284A30010060052505422A29D13
:1002B00094A3001005005250DE65F468B8B1001038
:1002C000F8B5C04610B5064C2378002B07D1054B76
:1002D000002B02D0044800E000BF0123237010BDB2
:1002E0000881022000000000D0910010044B10B5DE
:1002F000002B03D00349044800E000BF10BDC046F6
:10030000000000000C810220D091001070B50400A4
:1003100001238B40DDB2013DEDB2FF20002307E059
:100320008021490119435A00084E91530133DBB231
:100330001F2B09D82A001A40A242F1D05A000349C3
:10034000034850521800F1E770BDC04624810220D6
:10035000A0A0FFFF70B52C4B1B78012B48D0022BBF
:1003600049D0002B41D0052003F032F9274B186803
:100370008301A022D205944663441B69DB013DD46E
:10038000012252421000224B19688B01A025ED0575
:10039000AC4663441B69DB0101D5220008001D4BFC
:1003A00019688B01A025ED05AC4663441B69DB0190
:1003B00001D562000800184B19688B01A025ED05D6
:1003C000AC4663441B69DB0102D5620012190800C8
:1003D000431C09D08301A021C9058C466344986859
:1003E000201A801801380BD470BD80242402BAE78B
:1003F0008024E401B7E78024A401B4E70022C2E727
:10040000A0000138F0E7C046A48E02206C870220CD
:1004100070870220748702207887022070B501243B
:100420004C4B1C70FFF796FF4B4B18604B4B1A68F8
:100430009440A021C9054A4BCC509301A021C90585
:100440008C466344DB68DB01F7D4464B1A68012312
:1004500093400800424943509301A021C9058C46AE
:100460006344DB68DB01F7D43F4B1A6801239340F8
:1004700008003B4943509301A021C9058C466344C1
:10048000DB68DB01F7D4394B196801238B406046E8
:10049000334A83508B01A022D20594466344DA6824
:1004A00080235B0414001C401A42F3D1304D2A68AB
:1004B000303280239B01134301221A600021072060
:1004C00001F06CFF2A682B4B186804302A4B9A42C3
:1004D00000D008240019002101F060FF27490720FF
:1004E00002F0C8F81D4B186808F0E0FB1D4B1868B7
:1004F00008F0DCFB1C4B186808F0D8FB1B4B186895
:1005000008F0D4FB1A4C20681A4B196803680125BF
:100510002A008A409343036008F078FC184B1A685D
:100520001849206808F0BCFC2068174E0368326840
:100530009540AB4303600022316808F0FBFC316852
:10054000206808F063FC114B1A682068104908F015
:10055000A7FC70BD9C8E0220A88B02206C87022015
:1005600044040000708702207487022078870220EC
:10057000D4860220588E0220000020501D04001056
:10058000D0860220189300105C8E0220788E022004
:100590002004002070B50124484B1C70FFF7DAFEE0
:1005A000474B1860474B1A689440A021C905464B39
:1005B000CC509301A021C9058C466344DB68DB0164
:1005C000F7D4424B1A680123934008003E49435038
:1005D0009301A021C9058C466344DB68DB01F7D495
:1005E0003B4B1A680123934008003749435093015D
:1005F000A021C9058C466344DB68DB01F7D4354B89
:10060000196801238B4060462F4A83508B01A0223A
:10061000D20594466344DA6880235B0414001C40CE
:100620001A42F3D12C4D2A68303280239B011343A8
:1006300001221A600021072001F0B0FE2A68274B32
:1006400018680430264B9A4200D008240019002173
:1006500001F0A4FE2349072002F00CF8194B18689A
:1006600008F024FB194B186808F020FB184B186899
:1006700008F01CFB174B186808F018FB164B18689D
:10068000164B1968036801228A409343036008F0FF
:10069000BDFB154B1B78002B07D0144B1A680E4B73
:1006A0001868134908F0FCFB70BD104B1A680A4B20
:1006B0001868104908F0F4FBF6E7C0469C8E02204B
:1006C000A88B02206C87022044040000708702205F
:1006D0007487022078870220D4860220588E022058
:1006E0000000205095050010A78E0220D086022021
:1006F000649300104C93001070B50124494B1C709A
:10070000FFF728FE484B1860484B1A689440A02118
:10071000C905474BCC509301A021C9058C466344C1
:10072000DB68DB01F7D4434B1A68012393400800D0
:100730003F4943509301A021C9058C466344DB68BF
:10074000DB01F7D43C4B1A68012393400800384979
:1007500043509301A021C9058C466344DB68DB014B
:10076000F7D4364B196801238B406046304A8350DA
:100770008B01A022D20594466344DA6880235B048F
:10078000100018401A42F3D12D4B1A681100303175
:1007900080239B010B43012119602A4B1B68043302
:1007A00029498A4200D008201818002101F0F6FDDE
:1007B0001E4B186808F07AFA1E4B186808F076FA93
:1007C0001D4B186808F072FA1C4B186808F06EFA96
:1007D0001B4D28681B4B19680368012422008A40BE
:1007E0009343036008F012FB184B1A6828681849F5
:1007F00008F056FB174D2868174E0368326894407E
:10080000A34303600022316808F094FB3168286834
:1008100008F0FCFA114B1A682868114908F040FBEF
:1008200070BDC0469C8E0220A88B02206C870220DF
:100830004404000070870220748702207887022019
:10084000D4860220588E022000002050D08602203C
:10085000349300107C8E02205C8E0220788E022061
:100860003C04002010B5064B1B78022B00D010BDB5
:10087000044B1B681B6BDB07F9D5FFF73DFFF6E761
:10088000A68E0220D4860220F8B50500012800D1EA
:1008900063E1022800D163E1002800D15AE1012080
:1008A00008F00CFAE44C2060012008F007FAE34B52
:1008B0001860012008F002FAE14B1860012008F0EE
:1008C000FDF9E04B18602268DF4B0C2A00D94AE1A1
:1008D000DE490B40D20213430C229343043A1343E4
:1008E000DB4A1340DB4A1340DB4A13400122134327
:1008F000DA4A1340022293430E32934310321343D9
:10090000022D00D935E10C229343AA001343CB4AB0
:1009100012680C2A00D932E1CC491940D3020B43AA
:10092000CF4A1068CF4A12680432CF49884200D1BA
:100930002BE1082152183F2A00D928E1CB49194060
:10094000D3030B43C24A1340F822D2001343BB4ADD
:100950001168BD4A0C2900D91FE1BC480240C902F8
:100960000A430C218A4304390A43B9490A40B94968
:100970000A40B9490A4001210A43B8490A40022104
:100980008A430E318A4310310A43022D00D90AE10D
:100990000C218A43A9000A43A94909680C2900D9F6
:1009A00007E1AA481040CA020243AD490C68AD49AC
:1009B00009680431AC48844200D100E108200918DC
:1009C0003F2900D9FDE0A9481040CA030243A049CD
:1009D0000A40F821C9000A43994908689A490C2835
:1009E00000D9F4E0994C2140C00201430C2081431E
:1009F000043801439648014096480140964801401A
:100A00000120014395480140022081430E3081437B
:100A100010300143022D00D9DFE00C208143A800F3
:100A20000143884800680C2800D9DCE0874C0C4062
:100A3000C10221438A4807688A48006804308A4C0A
:100A4000A74200D1D5E0082400193F2800D9D2E000
:100A5000864C0C40C10321437D480140F820C00072
:100A6000014378480068784C0C2800D9C9E0774FDA
:100A70003C40C00204430C208443043804437448BF
:100A800004407448044074480440012004437348FF
:100A90000440022084430E30844310300443022D6E
:100AA00000D9B4E00C208443AD002C4362480568B3
:100AB0000C2D00D9B1E065482040EC0204436848A1
:100AC00007686848056804356748874200D1AAE08E
:100AD00008202D183F2D00D9A7E064482040EC03E2
:100AE00004435B480440F820C000044355480768AD
:100AF0005B48006884465B480068083085006544B0
:100B0000BF01A020C005844667443D605848786016
:100B1000BE603C614A4C2468A40164442560554F82
:100B2000C7196760A6602161444909688901614469
:100B30000D60514C04194C608E600A613E4A126887
:100B40009201624415604D498C4660445060966045
:100B5000D360F8BD80263602A1E68026F6019EE627
:100B60008026B6019BE6464B464AC421464803F020
:100B700069F8464B464AD221434803F063F8404B9C
:100B8000404AC421404803F05DF80021D2E6414BC1
:100B9000414AB6213C4803F055F8394B394AC42143
:100BA000394803F04FF8394B394AB231364803F02F
:100BB00049F8334B334AC421334803F043F800204B
:100BC000FDE6344B344AB6212F4803F03BF82C4B5A
:100BD0002C4AC4212C4803F035F82C4B2C4AD22146
:100BE000294803F02FF8264B264AC421264803F053
:100BF00029F8002428E7274B274AB621224803F08A
:100C000021F81F4B1F4AC4211F4803F01BF81F4B3C
:100C10001F4AD2211C4803F015F8194B194AC42168
:100C2000194803F00FF8002053E71A4B1A4AB6216F
:100C3000154803F007F8C0466C8702207087022031
:100C4000748702207887022010801F00FF87FFFF33
:100C50003FF8FFFFFFFFBFFFFFFFDFFFFFFF7FFF4B
:100C6000D4860220588E022000002050FF7FE0FF33
:100C7000000002200080FFFF0000FFFF0080FEFF59
:100C8000D091001094930010F09100103C9200104D
:100C9000B0930010809200107C93001010B50D4BA3
:100CA0001B78002B0CD1EFF3108472B60A4B1B7823
:100CB000002B06D0012B07D0022B08D084F310881C
:100CC00010BDFFF767FCF9E7FFF7A8FBF6E7FFF7B2
:100CD00013FDF3E79C8E0220A68E0220F0B5DE46BF
:100CE00057464E464546E0B597B004900D00039236
:100CF000059320AB1F7821AB1B789A4622AB1B785B
:100D0000994623AB1B889B4624AB1C78012C23D02F
:100D1000022C24D0002C1CD0039BEB18B34200D330
:100D200008E2534B0499994200D90BE2182F00D9DD
:100D30000AE251460F2900D908E24946052900D99F
:100D400006E2002900D105E2514410290ADD002005
:100D5000F1E18026B602DFE780267602DCE7802616
:100D60003602D9E7802292020021424804F0A2FF15
:100D7000414B1D60414B039A1A60414B1F70414B20
:100D800001221A70404B1C7000230598BB4207D209
:100D9000C25C3E49895C3E4AD1540133DBB2F5E77F
:100DA0003A4B52469B5C1A0005933A4B1A70052049
:100DB00003F0FCF804F0FEFE051C049B580004F050
:100DC000F9FE011C281C04F0DAFE8046324B334A3F
:100DD0001A60334D334E2E60300008F08DF82B68CA
:100DE000B3420ED00721002001F090F92A4B1A6877
:100DF0002C4B9A4207D00721012001F087F90026E9
:100E000008E00621EFE70621F6E7062101F07EF96A
:100E10000136F6B2BE4208D21F4B1A681C4B985DD1
:100E2000204B9A42F1D00721F0E71B4E0121306898
:100E300007F0FCFF02001C4B1860306853009B1841
:100E4000DB00D033C318802149010B438021090600
:100E50001960196003680432012191400B4303605B
:100E6000124908F001F8124B186000262EE0C04627
:100E700000E1F50500800020A08B02209C8B022061
:100E8000A58E0220A38E0220A48E0220D8930010EB
:100E9000848B0220A98E0220D486022000003050CC
:100EA0007C8E022000002050588E022034930010C7
:100EB000D0860220A84B9A5DA84B1968A84B1868E9
:100EC00000230093013308F06FF80136172EF1DD8F
:100ED000A44B1F68102200210AA804F0EBFE802614
:100EE00076020A96F8235B020B938023DB020C93B5
:100EF000C0231B030C9310220AA906A804F0E0FEED
:100F0000BA1C0337079B0493974B04990B40D201FB
:100F100013433F033B430793102206A90EA804F096
:100F2000CFFE119B0493914B049A13401E431196DC
:100F3000404604F067FE86B2002E00D1F6E0300095
:100F400004F038FE011C404604F013FE8721C90559
:100F500004F029FE04F056FEC3B21B0236041E4301
:100F60000E96109B0493824A1A40824B13431093AF
:100F70000F9B0493804A1A4080235B0413430F9312
:100F8000774B1A681100303180239B010B430121FC
:100F90001960724B18680430784B9A4200D1C7E050
:100FA0000823C018012101F0F9F96E4B1A686B4F44
:100FB0006B4B98460EAB39684046006808F02CF839
:100FC0006F4D0121286807F031FF6E4E30602A68AE
:100FD00043001B18DB00D033D318802149010B4399
:100FE00080210906196019601368043001218140CD
:100FF0000B4313605B46D8B24946FFF787F9624955
:10100000286807F031FF614B9A46186031682868FC
:1010100001230093002207F0C7FF316828680023EE
:1010200000934B46059A914607F0BEFF53461E6853
:10103000102200210AA804F03DFE80256D020A95C9
:10104000F8235B020B938023DB020C93C0231B036A
:101050000C9310220AA906A804F032FE33001F33B5
:101060001A00079B0493404B04990B40F60133434D
:1010700012031343079309990491CA00D2088021EF
:1010800089050A430992424A13400793102206A990
:1010900012A804F015FE102212A90EA804F010FEEA
:1010A000119B0493314B04990B404A46D2031343DE
:1010B0001193384A13408022D20413431193364AC5
:1010C000134011930E952000FFF7DEFB43461D6889
:1010D0003C682A680123A3409A4313432B60039A78
:1010E000013A696820001030012383400B42F8D197
:1010F0000434A4006251254B1A68224C204D0EABDB
:101100002168286807F088FF296820680A68012399
:1011100083409A4313430B600023204A1370204AF4
:101120001370204B02221A70012004E0002314E700
:10113000002336E7002017B0F0BCBB46B246A946F4
:10114000A046F0BD0020F6E70020F4E70020F2E71B
:101150000020F0E70020EEE7D8930010588E022020
:10116000D4860220D08602207F00FEFFFF7FF0FFA2
:10117000FFFF0AFE0000D101FFFFFFE0000020504A
:101180007C8E02205C8E02203C040020788E02209F
:10119000FFFFFF9F1FFCFFE3FF83FFFF9C8E0220EA
:1011A0009D8E0220A68E0220F0B5DE4657464E46A2
:1011B0004546E0B597B003900F001400049320ABB0
:1011C0001E7821AB1B789B4622AB1B789A4623AB3B
:1011D0001B88059324AB1D78012D23D0022D25D02B
:1011E000002D1BD03B19634500D314E2534B039AE7
:1011F0009A4200D917E2182E00D916E25B460F2B4F
:1012000000D914E25346102B00D912E2002B00D172
:1012100011E25B44102B0DDD0020FDE180239B02D9
:101220009C46DFE780235B029C46DBE780231B02B2
:101230009C46D7E7802292020021414804F03AFD03
:10124000404B1F60404B1C60404B1E70404B0122C6
:101250001A70404B1D7000230498B34207D2C25C41
:101260003D49895C3D4AD1540133DBB2F5E73A4B45
:101270005A469B5C9B463A4B5A461A70052002F030
:1012800095FE04F097FC071C039B580004F092FCA9
:10129000011C381C04F073FC8146324B9846324FD7
:1012A0001F60380007F028FE43461B68BB420ED083
:1012B0000721002000F02AFF2A4B1A682A4B9A4285
:1012C00007D00721012000F021FF002708E00621B8
:1012D000EFE70621F6E7062100F018FF0137FFB21D
:1012E000B74208D21F4B1A681C4BD85D1E4B9A425E
:1012F000F1D00721F0E71B4F0121386807F096FD78
:1013000002001A4B1860386853009B18DB00D0337A
:10131000C318802149010B43802109061960196017
:1013200003680432012191400B430360104907F028
:101330009BFD104B186000272AE0C04600E1F50530
:1013400000800020A08B02209C8B0220A58E022012
:10135000A38E0220A48E0220D8930010848B02203A
:10136000A98E0220D486022000002050588E022030
:1013700018930010D0860220B04BDA5DB04B19688C
:10138000B04B186800230093013307F00DFE0137BE
:10139000172FF1DDAC4B1E68102200210AA804F0C3
:1013A00089FC80277F020A97F8235B020B93802336
:1013B000DB020C93C0231B030C9310220AA906A87E
:1013C00004F07EFCF11C321D079B03939F4B039896
:1013D0000340C9010B43120313430793102206A9CC
:1013E0000EA804F06DFC119B0393994B039A1340D4
:1013F0001F431197484604F005FC87B2002F00D127
:1014000005E1380004F0D6FB011C484604F0B1FBAE
:101410008721C90504F0C7FB04F0F4FBC3B21B022B
:101420003F041F430E97109B03938A4A1A408A4B2E
:10143000134310930F9B0393884A1A4080235B0445
:1014400013430F937F4E32681100303180239B018C
:101450001943012008602D32FF32134380225200CD
:101460001A607F49063000F0C3FF0121072000F019
:1014700095FF3268724B186804307A4B9A4200D15B
:10148000C7E00823C018012100F088FF6E4B1A68DE
:101490006B4B99466B4E0EAB49460968306807F0B6
:1014A000BBFD0121306807F0C1FC02006E4F3860BF
:1014B000306853009B18DB00D033C31880214901EA
:1014C0000B43802109061960196003680432012169
:1014D00091400B430360654B52461343644A53816A
:1014E000644907F0C1FC644B98461860396830685D
:1014F00001230093002207F057FD3968306800236C
:10150000009353465A4607F04FFD43461B689846E2
:10151000102200210AA804F0CDFB80235B029A462A
:101520000A93F8235B020B938023DB020C93C02306
:101530001B030C9310220AA906A804F0C1FB424623
:101540000832079B0393414B03990B404146C90165
:101550000B43120313430793102206A912A804F0A9
:10156000AFFB102212A90EA804F0AAFB119B039353
:10157000374B039A13405A46D203134311933F4A01
:1015800013408022D2041343119353460E93109BB1
:101590000393304B039A1340109339680EAB4246C5
:1015A000306807F039FD2800FFF76EF932684B46C6
:1015B0001D6811680123AB4099430B431360013C44
:1015C000516828001030012383400B42F8D10435C4
:1015D000AD00AC50244B1C6811680123A340994313
:1015E0000B431360516820001030012383400B42ED
:1015F000F8D10434A400059BA3500023204A1370A3
:10160000204A1370204B01221A70012004E00023AD
:1016100005E7002336E7002017B0F0BCBB46B24612
:10162000A946A046F0BD0020F6E70020F4E7002020
:10163000F2E70020F0E70020EEE7C046D893001064
:10164000588E0220D4860220D08602207F00FEFF22
:10165000FF7FF0FFFFFF0AFE0000D101FFFFFFE068
:101660001D040010000020505C8E0220406000002D
:101670002804002020040020788E02201FFCFFE3B5
:101680009C8E02209D8E0220A68E0220F0B5DE46A2
:1016900057464E464546E0B591B080468B4616000B
:1016A0001C001AAB1D781BAB1B789A461CAB1B7831
:1016B00099461DAB1F78012F14D0022F16D0002F92
:1016C0000CD05B469B19634500D38AE1CA4B984511
:1016D00000D98EE1182D0DD9002083E180239B02D3
:1016E0009C46EEE780235B029C46EAE780231B02D0
:1016F0009C46E6E7802292020021C04804F0DAFA14
:10170000BF4B5A461A60BF4B1E60BF4B1D70BF4B8C
:101710004A461A70BE4B00221A70BE4B1F70002141
:1017200006E0635CBC4AD25CBC4B5A540131C9B27E
:10173000A942F6D3B84B52469B5C9A46B84B5246E8
:101740001A70052002F032FC04F034FA041C4346FF
:10175000580004F02FFA011C201C04F010FA8046F7
:10176000B04CB148206007F0C7FB0121206807F0AA
:101770005DFB0200AD4B1860206853009B18DB0036
:10178000D033C318802149010B4380210906196019
:10179000196003680432012191400B4303604B46FA
:1017A000002B06D0A24907F05FFBA24B1860002473
:1017B00011E0A14907F058FB9E4B1860F7E7964BE4
:1017C0001A5D9A4B1968974B1868002300930133F0
:1017D00007F0EAFB0134172CF1DD924B1A68924BAB
:1017E0009A4205D00721504600F090FC002406E004
:1017F0000621F8E7062100F089FC0134E4B2AC428E
:1018000008D2884B1A68854B185D874B9A42F1D0F5
:101810000721F0E74B46002B44D0864B1C68102272
:10182000002108A804F046FA80235B020893F823FD
:101830005B0209938023DB020A93C0231B030A93F4
:10184000102208A904A804F03BFAE21D059B0393AB
:101850007A4B03990B40E40123431203134305938E
:10186000102204A90CA804F02BFA0F9B0393744ACE
:101870001A4080235B0213430F93404604F0C2F9E1
:1018800084B2002C38D0200004F094F9011C4046AA
:1018900004F06FF98721C90504F085F904F0B2F965
:1018A000C3B22AE0634B1C681022002108A804F090
:1018B00001FA80235B020893F8235B0209938023DB
:1018C000DB020A93C0231B030A93102208A904A871
:1018D00004F0F6F9A21C0334059B0393574B0399BC
:1018E0000B40D2011343240323430593102204A980
:1018F0000CA804F0E5F9B8E700231B0224041C43FC
:101900000C940E9B03934F4A1A40A023DB0213430F
:101910000E930D9B03934C4B039A134052461206B1
:1019200013430D933F4C22681100303180239B01FB
:101930001943012008602D32FF32134380225200E8
:101940001A604249063000F053FD0121072000F0E3
:1019500025FD2268354B18680430334B9A423CD041
:101960000823C018012100F019FD324B1A682F4CD2
:101970002C4D0CAB2168286807F04EFB29682368C2
:101980000433294A91422AD008229B181F2213406F
:1019900001252A009A402E4B1A603800FEF774FF8A
:1019A000204B1A68214B1C681368A540AB431D43AC
:1019B0001560013E516820001030012383400B4226
:1019C000F8D10434A400A6500023224A1370224AFE
:1019D0001370224A1370012004E00023C1E70022A3
:1019E000D3E7002011B0F0BCBB46B246A946A046E2
:1019F000F0BD0020F6E7C04600E1F50500800020BC
:101A0000A08B02209C8B0220A58E0220A78E022094
:101A1000A38E0220A48E0220D8930010848B022073
:101A2000A88E0220D486022000002050588E02206A
:101A30004C930010D0860220649300107F00FEFFBC
:101A4000FF7FF0FFFFFF0AFEFFFFFFE0950500109C
:101A500080E200E09C8E02209D8E0220A68E022055
:101A6000024B187801235840C0B270479C8E022068
:101A7000F0B5DE4657464E464546E0B583B0814652
:101A80008C4693465A4B1B78002B22D1594B187821
:101A9000012839D002283BD0002831D0564B196894
:101AA000564B1B68C9184A1E554B1B689A4233D9BE
:101AB0005B1A4344013B534A1360524B1E68012892
:101AC0006ED002284AD0002800D18BE0484B01227A
:101AD0001A70484B1B785A461370474B1B68474A8D
:101AE00012689B184A461360464B62461B68136097
:101AF000454803B0F0BCBB46B246A946A046F0BD7F
:101B000080239B029846C9E780235B029846C5E77D
:101B100080231B029846C1E75B1A0133394A1360E0
:101B2000CBE73A4B995C023901238B402340891A59
:101B3000CB4018430132364B1B789342F1DC01361F
:101B40002860B04500D800260137BA45BED9B50097
:101B50002D4BED182C6800220020ECE700231F001D
:101B60008A46F2E7294B995C023901238B400340F6
:101B7000891A0B411F43BFB20132254B1B78934298
:101B8000F0DC01362F80B04500D800260134A24594
:101B90009CD973001C4A9D18D05A00220027ECE7FC
:101BA00000248A46F3E7194B185D0238012383406D
:101BB0002B40001B03411A43D2B20134144B1B7853
:101BC000A342F0DC01360A70B04500D80026013788
:101BD000BA4500D87AE70C4BF1189D5D019B0024B3
:101BE0001A00EBE7002301901F008A46F0E7C04689
:101BF0009D8E0220A48E0220A08B02209C8B0220AE
:101C0000A88B0220A48B022000800020848B02205D
:101C1000A58E022010B504F0E5F910BDF0B5D6464A
:101C20004F464646C0B588B006000F000792002414
:101C300006E01278552A10D07D4B00221A7001342C
:101C4000BC4200D3EDE07A4A15786B1CDBB213700E
:101C5000315D784A5155012BEBD0022B0FD0022B6E
:101C6000EDD906939A1E7348825CAA2AE7D15A1EC0
:101C7000825C552AE3D100220021884615E06D4A96
:101C80005278AA2AEBD06A4B00221A70D7E70132A9
:101C900068488446805C013DFF3D454060464146C2
:101CA000455401208446E04401320699914207DD03
:101CB000604DAD5CF02DEAD05E4841464554F0E7FA
:101CC0005C4A9278002A09D0012A13D007995A4811
:101CD000FFF7A0FF564B00221A70B0E7052B04D087
:101CE00007995548FFF796FFF4E707995348FFF720
:101CF00091FFEFE7524B534A13601B78012B33D00F
:101D0000022B5DD04B4D6B792F22AA5C91460922A4
:101D10009446AC442232A95CEA6A12020A43924613
:101D20002721685CA96A090201432320285C8046B8
:101D3000686A0002424610434A4603925A1E934183
:101D400002932B7901932123EB5C00936346524667
:101D5000FFF79CFC00285FD007993B48FFF75AFF2C
:101D60003A4B01221A70B5E7324D2E33EB5C092253
:101D70009446AC442232A95CEA6A12020A439046B5
:101D80002721685CA96A090201432320285C814657
:101D9000686A00024A4610430493EB7999462B7A0D
:101DA0001B024A46134303936B7902932B790193E9
:101DB0002123EB5C009363464246FFF7F5F9C9E740
:101DC0001C4D2D33EB5C09229446AC442232A95CB5
:101DD000EA6A12020A4390462721685CA96A09024E
:101DE00001432320285C8146686A00024A4610436A
:101DF0000493EB7999462B7A1B024A4613430393CB
:101E00006B7902932B7901932123EB5C009363465A
:101E10004246FEF763FF9DE707990D48FFF7FAFE7C
:101E200058E708B0E0BCBA46B146A846F0BDC04687
:101E30009B8E0220B08B022094920010A89200107A
:101E4000B38B0220448C0220C09200109E8E022090
:101E5000D492001010B582B00400002004F0D2F833
:101E6000431C0ED06B46D871002C02D0200002B06B
:101E700010BD002201216B46D81DFFF7CFFE0134B3
:101E8000F4E70024F2E710B50020FFF7E3FF10BDF0
:101E900010B50120FFF7DEFF10BD000070B584B063
:101EA00003AB02AA01A94B4800F0D8F8002803D1DF
:101EB0004849494801F060FF039A0299019800F0EF
:101EC00091F804F09BF8FA20800001F08FFA80224C
:101ED0000021424803F0EEFE192000F02FF9D02334
:101EE0001B06802292045A625A6122E0029B5B0028
:101EF0000293039B5B00039342E0029B9B000293CF
:101F0000039B9B0003933BE00134029B9C420DD258
:101F1000039B5A1C0392E85C03F0FEFF80239B02A4
:101F2000039A9A42F0D300230393EDE72C4B00224F
:101F30001A702B4B1B78002B48D0FFF791FD00281F
:101F400020D101AE02AC320003A92000FFF790FDC2
:101F50000500642001F04AFA207803F0DDFF607884
:101F600003F0DAFFA07803F0D7FFE07803F0D4FFA6
:101F7000642001F03BFA3378012BB7D0022BBCD0A0
:101F80000024C2E7D0231B06802292049A61FA2023
:101F9000800001F02BFAFFF77BFF00280AD0FEF744
:101FA0007DFE0F4B00221A70D0231B068022920464
:101FB0005A61BEE7D0231B06802292045A61FEF7C5
:101FC00051FCFA20800001F011FAB2E7FFF75BFF45
:101FD000AFE7C046400D0300E4920010B08B022032
:101FE0009E8E0220F0B583B004000D00160000F0B4
:101FF00029F9002801D003B0F0BD154F00973B0030
:1020000001220121053001F0CFFE00962B002200B5
:102010000121104801F0D0FF31006943200003F096
:10202000EDF904000C4B009300220221042001F082
:10203000BBFE0094230000220121052001F0B4FE24
:1020400000973B0002220021062001F0ADFED2E7FE
:10205000006CDC0200800240001BB700F0B5DE46D9
:1020600057464E464546E0B583B080468B460092C3
:102070000193042001F09AFFFA21890003F0BEF9D0
:102080008246A0235B0099462CE0013C002C20D026
:1020900025007D432900300003F0B0F94045F4D11C
:1020A0002900300003F0AAF90029EED173019B1B2F
:1020B0009B009E19F6005B461E60009B1F60019B03
:1020C0001C60012003B0F0BCBB46B246A946A04646
:1020D000F0BD013F002F01D03C00D7E701235B4258
:1020E0009C46E1444B460F2B09D956464B465E436E
:1020F000044BF218044B9A42F0D80727EAE7002075
:10210000E0E7C046508EF4FF50F80C0010B5830095
:10211000084A944663441C6840226240C02414402C
:102120008022520113431C60C000034B9C46604454
:10213000416010BD04C001400040014010B50123C2
:102140008340D0221206936293610521FFF7DEFFE0
:1021500010BD0000EFF3108072B6034B1B68002B1C
:10216000FBD0BFF35F8F70472C0100D0BFF35F8FB0
:10217000024B00221A6080F3108870472C0100D0B7
:10218000F8B506000C001500FFF7E4FFE308F718A8
:10219000F15C07222240012393400B4205D1DBB2C0
:1021A0000B433B70FFF7E2FFF8BD2100280001F070
:1021B000E3FDF0B583B00600019114001F00FFF7A6
:1021C000C9FF00E00134BC420CD8E308F518F35C09
:1021D0000721214001228A401A42F3D1D2B21A4388
:1021E0002A7001E001246442FFF7C0FF002C02DBEB
:1021F000200003B0F0BD019B002BF9D0089801F03E
:10220000BBFD000070B505000C00FFF7A3FFE3085D
:10221000EE18EA5C07210C400123A340134204D0CE
:102220009A433270FFF7A2FF70BD034B034A2C3173
:10223000034801F007FDC046F093001050940010D1
:1022400010940010034B1B6802201840431E984155
:10225000C0B2704700C00640002307E0054A9A1844
:102260009200BFF35F8F0021116001331F2BF5D95E
:102270007047C04640000034054A1078431CDBB26A
:102280001370172B02D9130010221A707047C04622
:102290004204002000B583B00100044B00931F23CB
:1022A00018220348FFF785FF03B000BD60940010BB
:1022B000D8860220074B9B68103080001950BFF36E
:1022C0005F8FBFF35F8F044B0021196082F310888A
:1022D0007047C04600ED00E0240100D010B5091A97
:1022E000081F0A4B9C466144094A914208D8C3071B
:1022F00006D440104005400D064B184380B210BD77
:10230000054B064A9921064801F09CFCFC07000099
:10231000FE0F000000E0FFFF7C940010D896001034
:10232000AC94001010B5091A04394C08090B08D1F7
:102330004905490D064A11430180064B234343805A
:1023400010BD054B054AA121054801F07BFCC046A4
:1023500000F0FFFF00F8FFFFE8940010AC960010BB
:10236000AC94001001238340034A10681840431EB8
:102370009841C0B27047C04600E100E0002904D097
:10238000034B1860034B18607047034B1860FBE762
:1023900080E200E000E100E080E100E010B5012310
:1023A00083401800FFF7EAFF10BD000001238340BF
:1023B000014A13607047C04600E200E0024B9B6890
:1023C00010308000C058704700ED00E010B5FFF7F6
:1023D000F5FF002805D0054BC01A2F2803D801208F
:1023E00010BD0020FCE70020FAE7C04644040020AE
:1023F00070B504000D00EFF3108672B60C4B1B682D
:10240000002BFBD0BFF35F8F2000FFF7D7FF094BF6
:10241000984201D0A84205D1320029002000FFF7E0
:1024200049FF70BD044B054A7C21054801F00AFCB8
:10243000240100D0CD010010F89400100C9700107A
:10244000AC940010F0B5DE4657464E464546E0B522
:1024500089B0814601911500EFF3108A72B6744B72
:102460001B68002BFBD0BFF35F8F724B0027DF5739
:10247000002F40DB7C00E419A4006F4824180622DA
:10248000A2566C4B1A706D4B9A684B4610339B00EA
:10249000D35898461E001B1A2F2B38D9684B9845E5
:1024A0002FD105AE674B33807B009B46D819800047
:1024B000614B9846404402306349FFF70FFF70803C
:1024C000624BB380FF23B371F571019B07935F44A7
:1024D000BF0047440ECE0EC701231C43A046524600
:1024E00041464846FFF7E6FE09B0F0BCBB46B2469F
:1024F000A946A046F0BD564B564ACD21564801F09C
:10250000A1FB564B534AD421534801F09BFBC043D7
:1025100040440C2102F072FF002912D101239E4396
:10252000B34633000026DA79AA4211D9062159565A
:1025300000290CDB4A00521892001E003E4B9B18EB
:10254000F1E7474B434AE021434801F07BFB1E0083
:10255000002E3BD005AB434A1A80813A5A800623AD
:10256000F3560293002B18DABD20000205AB9B4600
:102570009880029A9A71DD71019A0792301D2100AC
:10258000FFF7ACFEB080B7717B00DB199B002A4FD0
:10259000FF185B4607CB07C7A1E77800C01980008A
:1025A000254BC0180430321DB388D90A1C2907D125
:1025B0005B055915023149005118FFF78FFED5E729
:1025C000294B2A4AA721244801F03CFB05AE1D4BAC
:1025D00033807B000293D8198000174A904602008E
:1025E00042440392901C1849FFF778FE7080039ACA
:1025F000101D5946FFF772FEB0801D4B5A464146EA
:10260000521A524153431B0DB371F571019A07924F
:10261000029B9C466744BF0047440ECE0EC7114B39
:102620005A461380813B538001231C43A04656E742
:10263000240100D0A18E02204404002000ED00E01F
:10264000CD01001000A1FFFF7404002000BDFFFFBA
:1026500030950010F4960010AC94001058950010BE
:102660008095001001480000F4950010E4960010D9
:10267000AAAA0000F0B5CE46474680B583B0060052
:102680000D00EFF3108872B6564B1B68002BFBD081
:10269000BFF35F8F544B9A6834001034A300D758AF
:1026A000524B9F4207D0AF4200D199E00197504B67
:1026B000FB1A2F2B09D9424639003000FFF7FAFDEB
:1026C00003B0C0BCB946B046F0BD3000FFF74AFECB
:1026D000814600213000FFF761FEBFF35F8FFDF7F9
:1026E000C2FD002801D0844211D10123019C9C43EA
:1026F0000022A368AB4212D00622A256002A0DDBAC
:1027000053009B189B002200394CE418F1E72C2160
:10271000384B394AFF31394801F094FA2200AB4274
:1027200057D106256557002D39DB6B005B199A00E0
:102730002F4B9B189A68A260DA79E27106229A56AA
:10274000A2719B795BB2002B10DABD200002A08041
:102750006B005B199B00264AD318294A117899719E
:10276000157049463000FFF719FEA4E7201D6B00E5
:102770005B199B001E4A9B181A1D9B88D90A1C29AD
:1027800007D15B055B15023359005118FFF7A6FD11
:10279000DDE71C4B1C4AA721184801F053FA00281A
:1027A00012D1002A0ED0FF239371184B9380144A44
:1027B0001378A371164B0E49641A644163431B0DD1
:1027C0001370CEE7094FF2E7201D1249FFF7AAFD6B
:1027D000C7E76021104B084AFF31084801F032FA80
:1027E000024F68E7240100D000ED00E0CD010010A9
:1027F000440400200C960010C4960010AC94001005
:10280000A18E0220F4950010E496001000BDFFFF99
:10281000AAAA00007E0400203096001070B50400C3
:10282000012606432D4BF31A2F2B28D8FDF71BFD4D
:1028300000282BD0EFF3108C72B6294B1B68002BAD
:10284000FBD0BFF35F8F274D22002449521A52411B
:1028500055432D0D6DB2244B9B6880001B58B3422D
:102860001BD00022032A32D853009B189B001B491F
:10287000CB189B795BB2AB421FD00132F2E7C22189
:102880001A4B1B4A49001B4801F0DCF988211A4BFE
:10289000174AFF31174801F0D5F9134B9B68174AC7
:1028A0001A50174B1A78A2711D70BFF35F8F0C4B33
:1028B00000221A608CF3108870BD0800530099182C
:1028C00089004118FF268E710E4A8A80E9E7CC21E3
:1028D0000D4B074A4900074801F0B4F944040020B1
:1028E000240100D0AAAA000000ED00E038960010F4
:1028F00090960010AC94001060960010CD0100106E
:10290000A18E022000BDFFFF6C9600100022044B38
:1029100002E0044902C30132072AFAD97047C046CF
:1029200000E400E08080808000B583B00100D02307
:102930001B061B680648C018064B0093052300229F
:10294000FFF737FC002801DB1F23181A03B000BD76
:10295000948E022074960010024B9C4661448900BC
:10296000016070474000003470B505000C0008009D
:1029700000F0CCFD200000F0FFFE0849200000F030
:102980003FFEFFF779FC064B9C4660448000686080
:102990002C75A400034BE55070BDC046AD2C001053
:1029A00040000034348C02200A4B1A68EFF3108187
:1029B00072B61368002BFCD0BFF35F8F054B1B680A
:1029C000BFF35F8F00221A6081F3108840BF0020A0
:1029D00000217047548E022010B5002922D00368D0
:1029E0001B7B99421ED8174B9C46614409018368A2
:1029F0009C4661440C684968002A19D003681B7B17
:102A00009A4215D883680F488446624412019A1886
:102A100010685368020001208B4201D80ED00020BC
:102A2000C0B210BD084B094A3B21094801F00AF920
:102A3000054B064A3B21064801F004F9A242EFD8B3
:102A4000EDE7C046FFFFFF0F74970010309A0010AB
:102A50003C97001010B500291ED0037B99421BD86B
:102A60004B005B18033B0468A4466344002919D05B
:102A7000002A1DD0914221D0002A25D0047BA242F9
:102A800022D8046850008018033820188170197803
:102A900000291FD11A7010BD104B114A682111482E
:102AA00001F0D0F8104B114A6F310E4801F0CAF80E
:102AB0000F4B0E4A70210B4801F0C4F80D4B0B4A26
:102AC0007121084801F0BEF8044B054A6821054809
:102AD00001F0B8F841701A70DDE7C046A897001001
:102AE0009C9A0010C49700100C980010789A00105F
:102AF000189800102498001070B506000D001400FE
:102B0000002914D0002A14D08068736898470028E0
:102B100006D0220029003000FFF79CFF280007E0C4
:102B20002A0021003000FFF795FF200000E0100090
:102B300070BD0800FCE70000F0B583B0050000920E
:102B400001930AAB1C780BAB1F78002C26D00368CE
:102B50005A7B944207D10123002B19D1002C3BD181
:102B6000200003B0F0BD002C0CD01A7B944209D891
:102B70001A6863001B19033BD3189B78002BEBD01A
:102B80000123E9E73E4B3F4A68213F4801F05AF8EC
:102B90003E4B3F4A65213F4801F054F803689C7B57
:102BA000002CDBD012D01A7B94420FD8620012198D
:102BB000033A19688C46624451789973002900D110
:102BC000D9730023937053701370C7E72C4B2D4AB1
:102BD00068212D4801F036F8002C3AD02B681B7B79
:102BE0009C4236D82C4BE3181B01AA6894466344D8
:102BF000009A1A60019A5A60089A9A60099ADA60F3
:102C00002E68002C2BD030D0337B9C422DD8630013
:102C10001B19033B32689446634400229A705A7031
:102C20001A70717B22003000FFF766FF70738442D8
:102C300000D095E7287D009A019B00F029FD061E33
:102C400001D0002F17D00C9B002B00D188E71E70FD
:102C500086E7124B124A3B210E4800F0F3FF114B5E
:102C6000114AA521084800F0EDFF054B054A6821EF
:102C7000054800F0E7FF2868210000F031FFE2E797
:102C8000A89700109C9A0010C49700103C98001060
:102C9000A89A00103C970010FFFFFF0F74970010D8
:102CA000309A0010389700108C9A0010F0B5DE466C
:102CB00057464E464546E0B58BB009900023089331
:102CC0008200B24BD658370032E0B14BB14A3F21B7
:102CD000B14800F0B7FFB14BB14A3B21B14800F019
:102CE000B1FFB14BB14A8C21AE4800F0ABFFB04B05
:102CF000AE4A9021AB4800F0A5FFA84BAD4A402159
:102D0000A84800F09FFF2A686B68099800F0C0FC93
:102D100000239A4698467B68BFF35F8F00221A60B3
:102D200086F310884346002B51D1002800D126E1BC
:102D300000F0F8FB02000B1EC7DB0020002106900C
:102D400007917868EFF3108672B601680029FCD00D
:102D5000BFF35F8F396888464C7B002C32D0BAD0E5
:102D6000097B8C42B7D8944965182D01B9688C4607
:102D7000654428686968801A99410029C3DC01D13B
:102D80000028C0D10021404600F0A0FEA042A8D1FA
:102D90002A686B6806920793AB689846EB689A4678
:102DA0004346002BA3D0002CA7D03B681B7B9C4242
:102DB000A3D8631EFA68D35C08931B0218433861DA
:102DC0000020A8E700239A4698460020A3E7089B26
:102DD0001B022343994651461800C04705000E00C8
:102DE0007A68EFF3108B72B6136859424B41D9B22F
:102DF000002BF9D1BFF35F8F002E26DB002E52DDB2
:102E00003B69002B53D04B4572D100F08BFB020085
:102E10000B1E73DB0100180052197341984202D84F
:102E200004D1914202D901225242D317002B6BDB0D
:102E300000210491013103910294514601914146D0
:102E400000913800FFF778FE49E03B69002BD5D0B0
:102E50004B451CD1069A079B10001900521BB34129
:102E6000994202D804D1904202D901225242D3178A
:102E7000002B12DB00210491013103910294514691
:102E80000191414600913800FFF756FE27E04B4B79
:102E9000464A9F21434800F0D5FE3D4B3D4A3F2125
:102EA0003D4800F0CFFE002E01D1002DA8D13A6898
:102EB000002C45D0537B9C422CD1012100293FD1CD
:102EC000D37B002B42D1D473002C52D03B681B7BA8
:102ED0009C424ED8FA68013C135D01331355002320
:102EE0003B617A68BFF35F8F13608BF310881FE735
:102EF000324B2E4AA2212B4800F0A4FE244B254A37
:102F00003F21254800F09EFE214B224A3F212248C6
:102F100000F098FE002C0DD0137B9C420AD8630071
:102F20001B19033B1068844663449B78002BC5D073
:102F30000121C3E7224B234A6821234800F082FE87
:102F4000224B234AF621204800F07CFE002B0AD0B9
:102F5000117B8B4207D85900CB18033B11688C4674
:102F600063445C70AFE7164B164A6821164800F0C0
:102F700069FE0A4B0F4A40210A4800F063FE0BB07D
:102F8000F0BCBB46B246A946A046F0BD348C022038
:102F900064980010FC99001080980010749700103D
:102FA000309A00103C970010C4980010149A00103A
:102FB000DC980010549A0010FFFFFF0FE8980010F3
:102FC000A89700109C9A0010C49700102499001034
:102FD000689A001010B50A4B5B68002B04D00A21D8
:102FE0000848FFF7B9FC10BD054C2300064A102124
:102FF000206800F08BFC03212000FFF7B5FCEEE712
:103000008C040020548E0220D929001010B5064BE4
:103010005B68002B01D0044810BD044B044A5C21BE
:10302000044800F00FFEC0468C04002048990010B0
:103030003C9A00103C970010F0B5DE4657464E46CD
:103040004546E0B58BB0804616001F00149B9A469B
:10305000159B994616AB1B789B461F2302AA9446E4
:10306000634400221A7032E0002809D042461268F8
:10307000127B904204D8421E4146C9688A5C48E0EF
:10308000434B444A4021444800F0DCFD0798002BA4
:1030900075D05B46002B72D04946D04704000D0026
:1030A00003000B4300D171E0002946DB00F03AFA3F
:1030B00006000F1E55DB36196F41B94202D804D104
:1030C000B04202D901267642F717002F4FDB434664
:1030D0005A68EFF3108472B6136859424B41D9B263
:1030E0000791002BF8D1BFF35F8F1F3302AA9446DC
:1030F000634404930023039302934B460193534686
:10310000009332003B004046FFF716FD031EABD193
:10311000020041464968BFF35F8F00250D6084F3CC
:103120001088002B29D01F2302A98C4663441B78EA
:10313000002BABD112021043A9E732003B00361B33
:10314000AF41BB4202D804D1B24202D90126764235
:10315000F717002FBBDA114B114A3F21114800F03D
:1031600071FD0E4B0E4A3F210E4800F06BFD0B4BDC
:103170000B4A3F210B4800F065FD012040420BB097
:10318000F0BCBB46B246A946A046F0BD0798F6E79C
:1031900074970010549A00103C9700106498001027
:1031A000FC99001080980010F8B504004268EFF315
:1031B000108572B6136858424341D8B2002BF9D13A
:1031C000BFF35F8FCBB22268567BB3421BD1012085
:1031D000002848D0206988422BD0090AC9B2002BA8
:1031E0002ED02068007B83422AD8581EE668305CC7
:1031F00088422BD000206368BFF35F8F00221A60E3
:1032000085F31088F8BD002B0DD0167BB3420AD889
:103210005E00F618033E1768BC466644B678002E7A
:10322000D6D00120D4E7134B134A6821134800F08D
:1032300009FD8521124B134A4900134800F002FD95
:10324000124B134A4021104800F0FCFC19001000FA
:1032500000F046FC0028CED112210E4B094AFF3166
:10326000094800F0EFFC23698B42C4D1002323619D
:10327000C1E7C046A89700109C9A0010C4970010A0
:103280006C990010E49900103C970010749700109E
:10329000549A001090990010F0B587B006000F0006
:1032A000FCF7E1FF00281FD106246442E517A419AA
:1032B0007D41BD4202D803D1B44201D9002400258A
:1032C000002D14DB0494059500F02CF902000B1E70
:1032D00013DBA41A9D41002D17DC14D030003900F7
:1032E00000F02CF907B0F0BD234800F045FD234B5A
:1032F000234A3F21234800F0A5FC204B204A3F21D0
:10330000204800F09FFC002CE8D0FFF77FFE002350
:10331000029301931C4B0093049A059BFFF78CFECC
:10332000002818DADAE7002300E00023002BD5D1CB
:10333000164B1A68EFF3108172B61368002BFCD09D
:10334000BFF35F8F114B1B68BFF35F8F00221A60C2
:1033500081F3108820BF0499059A0D4B5B6A9A424D
:10336000E3D80B48806A884203D29A42DBD001231B
:10337000DCE70123DAE7C046949900106498001056
:10338000FC99001080980010A9290010548E02208A
:1033900000400540F8B504000D0000F0C3F802003D
:1033A0000B1E10DB20002900801859418B4202D8E7
:1033B00004D1824202D901204042C117002908DB12
:1033C000FFF76AFFF8BD064B064A3F21064800F0AA
:1033D00039FC034B034A3F21034800F033FCC0464D
:1033E00064980010FC9900108098001010B5FA2223
:1033F00092000023002102F09FFBFFF7CBFF10BDDE
:1034000070B584B006000C00FFF700FE00230293A5
:103410000193194B009332002300FFF70DFE051EA8
:1034200011DD20BFFFF7F2FD2900FFF7BDFE134BB2
:103430005B6A9C421BD8114A926AB2421AD29C42E1
:1034400013D0012014E00D4B5B6A9C4209D80B4A53
:10345000926AB24207D29C4201D0012008E00020CB
:1034600006E0002004E0012002E0002000E000204F
:1034700004B070BD0120FBE7A92900100040054001
:1034800070B5EFF305833F2018401038EFF3108C30
:1034900072B6194B1B68002BFBD0BFF35F8F012363
:1034A00019008140154A5163154A12781400C4402E
:1034B000234214D0114B5C6A8300124D5B599C422D
:1034C00006D38300104C1B598A430D490A7007E04C
:1034D0000A4A031D9B0099589950002300E00023DD
:1034E000BFF35F8F044A002111608CF31088002B1A
:1034F00000D0984770BDC046280100D0004005406C
:10350000AC8E0220688E0220C085022010B501001A
:10351000024A0348FEF734FE10BDC046C09A0010B0
:103520009F8E0220044B5B6A034A906A1900536A1B
:103530009942F9D17047C04600400540084B5B6A8C
:1035400001E0074B5B6A8B42FBD301E0044B5B6AF3
:103550008B4203D1024B9B6A8342F7D37047C0462C
:103560000040054070B504000D00FFF7DBFF0200CE
:103570000B0020002900801859418B4202D804D149
:10358000824202D901204042C117002902DBFFF725
:10359000D5FF70BD024B034A3F21034800F052FBA8
:1035A00064980010649B00108098001010B50028EB
:1035B00007DB064B9A6A054B9B6A9B1A8342FAD338
:1035C00010BD0021FFF7CEFFFAE7C04600400540DE
:1035D00010B50A4B984207D843011B1A9B001818D4
:1035E000C000FFF7E3FF10BDFA2292000023002184
:1035F00002F0A2FAFFF7B6FFF5E7C0469BC4200031
:1036000070B504000D00EFF3108672B61B4B1B68FB
:10361000002BFBD0BFF35F8F002D1CD02000FEF7E6
:10362000CDFE174B83420BD019002000FEF7E0FEC1
:1036300001212000FEF7B2FE0123A340114A1360CE
:10364000A400114BE550BFF35F8F0C4B00221A60B2
:1036500086F3108870BDA2000B4B0021D1500122CF
:10366000A2400A490B7893430B7005492000FFF7ED
:1036700001F800212000FEF791FEE4E7280100D0C8
:103680008134001038600540C0850220AC8E0220D5
:10369000F0B5DE4600B584B00400150001921E00AE
:1036A0000293FFF73FFF03958E4202D84ED1854229
:1036B0004CD9EFF3108B72B6274B1B68002BFBD055
:1036C000BFF35F8F254A17780125A540EBB23B4336
:1036D0001370234B5D63221D92000199D150A2000B
:1036E0002049029850501B6A2B4212D11C4B1B6C74
:1036F0002B4208D00020BFF35F8F174B00221A60C7
:103700008BF3108823E0184B184AC121184800F0A9
:1037100099FAFFF707FF8E4214D802D1039B834228
:1037200010D80E4B1B78BB420ED00D4B1D625D6353
:103730001F2004400123A3400E4A1360074B1F7053
:103740001E38D8E70020D6E70120D4E7012004B0D6
:1037500080BCBB46F0BDC046280100D0AC8E022024
:1037600000400540688E0220E49A0010489B00103B
:10377000089B001080E200E0EFF3108C72B60B4B58
:103780001B68002BFBD0BFF35F8F01238340084AE7
:10379000136208490A789A430A70BFF35F8F034B9C
:1037A00000221A608CF310887047C046280100D0B0
:1037B00000400540AC8E022010B500291ED0037BCE
:1037C00099421BD84B005B18033B0468A446634432
:1037D000002919D0002A1DD0914221D0002A25D0DD
:1037E000047BA24222D804685000801803382018B5
:1037F0008170197800291FD11A7010BD104B114A21
:103800006821114800F01EFA104B114A6F310E4822
:1038100000F018FA0F4B0E4A70210B4800F012FA14
:103820000D4B0B4A7121084800F00CFA044B054A75
:103830006821054800F006FA41701A70DDE7C046BD
:10384000A8970010689C0010C49700100C980010F6
:10385000549C0010189800102498001070B50600B1
:103860000D001400002914D0002A14D08068736859
:103870009847002806D0220029003000FFF79CFF5F
:10388000280007E02A0021003000FFF795FF200004
:1038900000E0100070BD0800FCE7000010B5002338
:1038A000437301338373037BC3730123027B9A4207
:1038B00014D9002B0CD0027B934209D85A00D2189D
:1038C000033A01688C4662440133DBB25370EDE782
:1038D0000B4B0C4A68210C4800F0B4F9002A09D0BF
:1038E000924207D8016853009A18033A8A180023B5
:1038F000537010BD024B034A6821034800F0A2F93F
:10390000A8970010689C0010C497001010B50173B0
:1039100042608360FFF7C2FF10BD000070B5040075
:10392000081E00D170BD002934D0237B994231D8C4
:103930004B005B18033B2268944663445A78002A84
:10394000F0D02DD0237B9A422AD853009B18033BFA
:1039500021688C4663445D7800215970002825D089
:10396000237B984222D843001B18033B21688C46D6
:1039700063440021597001002000FFF76FFF06002B
:1039800029002000FFF7CAFF020031002000FFF7E6
:1039900065FFC7E7084B094A6821094800F052F95A
:1039A000054B064A6821064800F04CF9024B034AD1
:1039B0006821034800F046F9A8970010689C0010A1
:1039C000C497001070B505000C001600002928D01F
:1039D0002DD0037B99422AD84B005B18033B026829
:1039E000944663445A78002A27D19A78002A2AD12B
:1039F0001978FFF793FF0300002E03D0EA7B002A1B
:103A000027D1EC73002B37D1002C49D02B7B9C4263
:103A100046D82B6861000C19033C1C190023637005
:103A200070BD224B224A3821224800F00BF9224B6C
:103A3000224A6821224800F005F9224B1C4A3A210B
:103A40001C4800F0FFF8204B194A3B21194800F0B0
:103A5000F9F8002A0AD0297B8A4207D851008A182F
:103A6000033A29688C4662445470CAE7124B134AE1
:103A70006821134800F0E6F8002B0BD02A7B934214
:103A800008D843001B18033B2A689446634400226D
:103A90009A70B9E7084B094A6821094800F0D2F842
:103AA000054B064A6821064800F0CCF87C9B0010C4
:103AB000409C0010849B0010A8970010689C001088
:103AC000C4970010BC9B0010E49B001070B504006C
:103AD0000A00457B2900FFF775FF6073280070BD61
:103AE00070B50400002967D0437B8B420ED00029BB
:103AF00011D0037B99420ED84B005B18033B026840
:103B0000D0188378002B0CD1002056E00121FFF75C
:103B1000DDFF012051E0294B294A6821294800F0A6
:103B200091F8002B20D0227B93421DD85A00D31845
:103B3000033B2268D2182568EB5C8B421AD0002B1D
:103B40001BD0227B934218D85A00D318033B22681B
:103B5000D21853788B4216D0002BF0D11A4B1B4A47
:103B600067211B4800F06EF8144B154A6821154870
:103B700000F068F84378137007E0104B104A682192
:103B8000104800F05FF8437853700023837043704F
:103B900001222000FFF716FF0200617B814205D061
:103BA0002000FFF75BFE6073012006E0094B074A27
:103BB0006D21074800F046F8002070BDA89700105E
:103BC000689C0010C49700106C960010289C001090
:103BD000849B0010089C001010B50400FEF74CFBFD
:103BE00001002000FEF7B8FEFF232371BFF35F8FB3
:103BF00010BD10B50400FEF73FFB01002000FEF7EA
:103C0000ABFEFF23237100236371BFF35F8F10BDF1
:103C1000034B9C46614489000160BFF35F8F70478E
:103C20004000003410B504000120FEF733FB010012
:103C30002000FFF7EDFF10BD00BEFDE710B5FFF758
:103C4000FBFF000010B582B00C001900002A0CD058
:103C5000084B002A0BD00192009323000200064873
:103C600002F0C0F90120FFF7E7FF044BF1E7034A38
:103C7000F1E7C0463C9D00104C9D0010BC92001026
:103C800070B52B4B2B4A1A602B4B2C4A1A602C4BCD
:103C90009A682A4B9343FAD12A4C01E008CC984702
:103CA000294B9C42FAD300F001F9234B274A1A60B2
:103CB000234B9B68DB43DB01FAD1254B40229A67FB
:103CC0005A671A67DA66234C09E0234B234A83219B
:103CD0002348FFF7B7FF2000FFF77EFF0834214B92
:103CE0009C4209D22368002BF5D0012BEDD1200096
:103CF000FFF77FFF0834F2E71B4CA1681B4DC02281
:103D0000280001F0DDFFA560FCF7ADFA002800D027
:103D100000BEFEF7A1FAFEF7F9FDFFF75BF9144CC0
:103D200001E008CC9847134B9C42FAD370BDC046C3
:103D300000E00040BFCDFBFE00F00040FE7F3C00F5
:103D400000C000403005002040050020FFFFFF01BB
:103D500000F00140200500207C9D0010F09D001027
:103D60009C9D00103005002000ED00E000000020C8
:103D700040050020480500200FB400B583B0084876
:103D800002F0FEF8049B002B07D005A90191180052
:103D900002F006F9034802F0F3F80120FFF74CFFA8
:103DA000DC9D0010EC9D0010F8B5DE4657464E46EF
:103DB0004546E0B505000F0092460A9A93424ED35D
:103DC0001A0E91461E020A9A00233000494601F05D
:103DD00057FB80466C006419A4002F4B9C4664443A
:103DE0006368834200D260602B1FDBB29B46012BCD
:103DF0003BD9C0239B012343802212011A60AB00F0
:103E0000264A9958002905D0506901F0F7FA013087
:103E10000138FDD153465A0123685A40E0231A4025
:103E200080235B0123431A605A46012A28D9802344
:103E30009B012343802212011A604346636042467D
:103E400000233000494601F01BFBAD00134B5851D5
:103E50000120F0BCBB46B246A946A046F8BD104BB7
:103E6000104A2D211048FFF7EDFE012FC1D1C023CC
:103E70009B01234303221A60A368DB07FCD5C9E733
:103E80002168794003220A401A60A2680123BB40DE
:103E90001342FAD0CBE7C04600800040DC86022007
:103EA000009E0010589E0010149E001030B583B084
:103EB0000C2000F021F9FEF7C5F900280DD00023F1
:103EC00004E099002D4A2E4888500133092BF8D977
:103ED0002A4B2C4A5A6203B030BD2B4B00229A6702
:103EE00000F07CF9294B01221A60274B5B6C012BF7
:103EF000FBD1274B03221A60234B9B6B012BFBD179
:103F0000013300930433234A0121234800F054F87D
:103F100005230093214A0121214800F04DF8214B4F
:103F20000093002202210420FFF73EFF1E4D009562
:103F30002B00002201210520FFF736FF104C0094D2
:103F40002300002200210720FFF72EFF009423000A
:103F5000002200210820FFF727FF0A4B00932300CF
:103F6000002200210920FFF71FFF00952B000022EF
:103F700000210620FFF718FFADE7C046DC860220CF
:103F8000006CDC021BB70000008000403CB0004029
:103F900030B00040002F685900800240008C8647F6
:103FA00000C00240001BB700405973078000014B5E
:103FB000C0587047DC860220F0B5C64600B5040044
:103FC0000F0090461D000C2001F018FA06003D4A33
:103FD00042443D4B9A4243D843011B1A9901C91AE6
:103FE000C90009188901404601F008FA0200103A98
:103FF00098235B009A4239D86B1E062B3CD8069B4F
:10400000013B062B38D8069B9D423BD343461A09F9
:10401000B2423DD32D04069B1E0335432368002B7B
:104020003CDB2A4B9C424AD080225201284B1A602A
:10403000284B1A60284B9B6811009943FAD12760DE
:10404000A060231DC02292011A432123136023681C
:10405000002BFCDAE5600823136080BCB846F0BD95
:104060001E4B1F4A11211F48FFF7ECFD1E4B1C4A37
:1040700019211C48FFF7E6FD1C4B194A1C21194861
:10408000FFF7E0FD1A4B164A22211648FFF7DAFD2A
:10409000184B134A25211348FFF7D4FD22683F230C
:1040A0001340BB42BDD1A3681B051B0D8342B8D191
:1040B000E368EE22D2021340AB42B2D1CDE78022B8
:1040C0009201B3E780E84BD380F8A93200C00240E8
:1040D00000E0004000F0004000C00040689E00107A
:1040E000A09F0010C89E0010049F0010209F001089
:1040F0006C9F0010849F001080239B000343014AA3
:10410000D362704700800540024B1A68024B5A6028
:104110007047C046AC8B02200080054010B50200FD
:10412000164B8020C0051860154B164818600029F2
:104130000AD0154BE021C9041960002A09D1124B9D
:10414000802212061A6010BD0C4BE021C9041960D0
:10415000F3E753019B1A9800801800010B4B18607D
:1041600080235B04984202D3084B094A1A60FFF788
:10417000CBFF054B8022D2051A60E4E700B0054072
:1041800008200140FCFF010000A00540AC8B02208C
:10419000FFFFFF0010B5030010000C4A8024E40567
:1041A0001460002B0DD001221343094A094CD4613D
:1041B000094C5C401462516293620021FFF7AEFF2C
:1041C00010BD034B0022DA61F7E7C04600B005409E
:1041D00000800540D3C007B02D3FF84F064BAA2200
:1041E00012011A602F22DA60044B054A1A60024B52
:1041F0005B68002BFBDA7047004002400060024021
:1042000000B0FA00704710B5002802D00B6849686A
:10421000984710BD0100002007E083001B185B00D9
:10422000501C08601078C01830380A681378303B8A
:10423000DBB2092BF1D97047F0B5DE4657464E4642
:104240004546E0B583B093461F000C9B9A460D9CF3
:104250000E9B99460F9B9B0703D0B8460F000600A4
:1042600022E00192A34688464E46B9460700B44272
:1042700007D2551C4B4641462020B84701342A003E
:10428000F5E73D004F465C46019B9B46B1464646DE
:10429000B84637002E0007E0013C551C5346185D18
:1042A00043463900B0472A00002CF5D135003E00C6
:1042B00047460F9B9B0707D4100003B0F0BCBB46DA
:1042C000B246A946A046F0BDB0464E46B9462F00BC
:1042D0005D46531BB342EFD2541C4B46414620204F
:1042E000B8472200F5E7F0B5CE46474680B585B021
:1042F000944698460C9D0D9C0EAB1B789946109ADF
:10430000119B129EB7071CD4002B0CD0F7070AD5BF
:104310004F46002F02D10C37374204D0013B02E058
:1043200030272F550134944201D21F2CF8D9F707BA
:1043300007D59C4205D21F2C03D830272F550134B6
:10434000F5E7F70615D5770505D4002C03D0944280
:1043500024D09C4222D00F9A102A2BD00F9A102AD8
:1043600030D00F9A022A35D01F2C02D830222A557D
:1043700001341F2C05D84A46002A31D02D222A5557
:104380000134039602930194009543466246FFF779
:1043900053FF05B0C0BCB946B046F0BD621E012C4B
:1043A00006D00F9F102F01D01400D4E7023CD2E7B3
:1043B0001400D0E7B206D1D41F2CCFD878222A55CA
:1043C0000134D1E7B206CCD51F2CCAD858222A55C1
:1043D0000134C9E71F2CC7D860322A550134C3E71E
:1043E000720703D52B222A550134CAE73207C8D5F4
:1043F00020222A550134C4E7F0B5DE4657464E4622
:104400004546E0B593B081468A46089209931CABB5
:1044100010CB1B789B461E9D219B9846002C03D1F8
:10442000102342469A4390468023DB0046461E40B6
:1044300042461A4212D0002C22D000260EE0303321
:10444000D9B2771C0AAB99552900200000F0D6FF9D
:10445000AC4216D31F2F14D83E00040029002000C0
:1044600000F0CCFFCBB2092BE9D94246920605D524
:104470004121C918C9B20A39C9B2E2E76121F8E796
:10448000270043460693209B05931F9B04930395A7
:104490005B46029301970AAB0093099B089A514629
:1044A0004846FFF720FF13B0F0BCBB46B246A94612
:1044B000A046F0BDF0B5DE4657464E464546E0B54F
:1044C00095B0089009910A920B931E9E1F9C20ABF9
:1044D0001B789B46229B9946239D269B9A46330038
:1044E000234303D1103352469A4392468023DB0084
:1044F00057461F4052461A4219D0330023432DD04D
:10450000002714E03033DAB27B1C98460CABDA5546
:104510004A462B003000210000F0B2FFA5421FD810
:1045200019D043461F2B1BD8474606000C004A46AD
:104530002B003000210000F0A3FFD3B2092BE1D9FA
:104540005246920605D54122D218D2B20A3AD2B2C8
:10455000DAE76122F8E7B145E3D901E000239846A4
:1045600053460693259B0593249B04934B46039344
:104570005B460293434601930CAB00930B9B0A9A54
:1045800009990898FFF7AFFE15B0F0BCBB46B246DC
:10459000A946A046F0BD0000F0B5DE4657464E469F
:1045A0004546E0B591B083468A460C9298461A9CDF
:1045B00008941B9D099522002B002000290001F082
:1045C000DEF9002800D0E5E001225242D74B20005E
:1045D000290001F0CFF9002800D0DBE0012252428F
:1045E000D34B2000290001F0AFF9002800D0D1E022
:1045F00000220023089E3000099D290001F0A4F943
:10460000002800D0DDE008980999069007918023E2
:10461000DB001E9A1A400D921E9A1A4201D10623FF
:104620001C930698079904000D000A000600024337
:1046300000D1D1E0080D4005400DBE4CA4466044B9
:104640000A03120BBC4B13431F0001F0ABF9BB4A2A
:10465000BB4B01F03AF9BB4ABB4B01F017F9040020
:104660000D000022B94B3000390001F00AF9B84AB8
:10467000B84B01F02AF902000B002000290001F0DC
:1046800005F901F0A7F9814601F08CF904000D004D
:10469000B14AB24B01F019F90022B14B01F0F6F822
:1046A00001F098F90600AF4AAF4B2000290001F055
:1046B0000CF904000D00300001F074F9AB4AAC4B6A
:1046C00001F003F902000B002000290001F0D9F8E5
:1046D00004000D0002000B0001F0F7F80A900B91A6
:1046E000A44BF31800261F0522002B0020002900F0
:1046F00001F0CCF80E900F9122002B0000208021B9
:10470000C90501F0BEF804000D0000229A4B0A987A
:104710000B9901F0C0F80022984B01F0B7F80200A5
:104720000B000A980B9901F0B6F80022944B01F0A7
:10473000ADF802000B000A980B9901F0ACF80200EA
:104740000B002000290001F0A1F802000B000E98D8
:104750000F9901F0A0F80022774B01F097F8320092
:104760003B0001F0B2F806000F0004000D00069AAD
:10477000079B01F0FFF8002830D001235B429C46E4
:10478000E14400227D4B3000390001F084F8040040
:104790000D0023E01E9B04931D9B03931C9B02931F
:1047A000089A099B0092019343460C9A5146584639
:1047B00000F0FCF811B0F0BCBB46B246A946A046DA
:1047C000F0BD0023002406930794069680231B0661
:1047D0009C46654407951AE7002399464B46633388
:1047E000C62B1ED804261E9B1B0526D52B00234353
:1047F0000FD0644A644B0698079901F0B3F800287B
:1048000079D00022614B0698079901F09DF80028A5
:1048100071D01C9B4B4506DD4A46981A431E1C93DB
:1048200003E00526DFE700231C938023DB001E9AAC
:104830001A431E920026002399461D9B9E4264D275
:104840009F1B02231E9A1A400A921E9A134202D0FC
:10485000002E00D000274B46002B07D022002B0053
:104860000698079901F017F8069007910022002397
:104870000898099901F068F8002848D1444B1E9A1D
:104880001340049303971C9B0293069B079C009381
:10489000019443460C9A5146584600F087F8002E82
:1048A00000D187E71E9B9B063DD54525441C43460A
:1048B000020051462800D8474B46DA179B18534050
:1048C00005220592013E0496002203920A320292CA
:1048D0004A46D00F01900093434622005146584665
:1048E000FFF78AFD0A9B002B00D163E702005F46B9
:1048F0000C9E1D9D54E01C9B002B9ED00D9B002BFD
:104900009BD01C9B013B1C9397E7002799E7069CD3
:10491000079D2200290080200006844661440B0088
:1049200006920793AAE76525C0E7C046FFFFEF7F21
:10493000FFFFEFFF01FCFFFF0000F03FFB799F50FE
:104940001344D33FB3C8608B288AC63F0000F83FAA
:1049500061436F63A787D23F71A379094F930A40E0
:104960000000E03F1655B5BBB16B0240EF39FAFECF
:10497000422EE63FFF03000000002C4000002440D0
:10498000000018402D431CEBE2361A3F80842E4174
:10499000FFF7FFFF541C434651462020B847220032
:1049A000931BAB42F6D3100004E7C046F0B5DE46D9
:1049B00057464E464546E0B595B00690079193465A
:1049C0009946209F1E9A1F9B1000190000F0D7FFE8
:1049D000002831D101225242BF4B1E981F9900F08E
:1049E000B3FF002837D101225242BC4B1E981F99B9
:1049F00000F0C0FF00283DD10022B94B1E981F993E
:104A000000F0B8FF002850D10022B64B1E981F9925
:104A100000F09AFF002848D1002200231E981F9919
:104A200000F092FF002850D100239846229B5B059E
:104A300000D4B6E0002458E0229B0393219B02930C
:104A400003230193A84B00934B465A4607990698B7
:104A5000FFF7F2FB0EE1229B0393219B02930423B9
:104A60000193A24B00934B465A4607990698FFF7CD
:104A7000E3FBFFE00423229A1A4022990B4210D054
:104A80009B4B002A0FD00422229903912199029175
:104A9000019200934B465A4607990698FFF7CCFBC4
:104AA000E8E0944BEDE70322EEE7229B0493219B81
:104AB000039302971E9B1F9C009301944B465A46FA
:104AC00007990698FFF768FDD4E01E9A1F9B002007
:104AD000002100F0D6FE1E901F9101239846A5E705
:104AE0000CAB30221A55013F01341F2C01D8092F7D
:104AF000F6D81E981F9900F06DFF050000F052FFD8
:104B000002000B001E981F9900F0BBFEFA007A4BC2
:104B10009B181A685B680A920B9300F0D6FE089007
:104B2000099100F07BFF060000F038FF02000B0047
:104B30000898099900F0A5FE0890099100226F4B92
:104B400000F018FF00282ED00136300000F026FFBC
:104B500002000B000A980B9900F0FCFE002801D01F
:104B600001350026002F2CD1280000F01BFF020089
:104B70000B001E981F9900F084FE06000F00002213
:104B80005E4B00F0E1FE002846D100225B4B300076
:104B9000390000F0EFFE00283ED1EB073CD501358F
:104BA0003AE0062746E70022544B0898099900F09E
:104BB000CBFE0028D6D1002E01D0F307D2D5013686
:104BC000D0E7AA461F2C11D8013F0A21300000F07F
:104BD00015FC651C30310CAB19550A21300000F072
:104BE0000DFC092E0ED906002C00EBE755461F2CB4
:104BF0000CD87B1E002F09D00CAA302111551F00A4
:104C00000134F4E72B0055461C00F0E71F2C03D8B5
:104C10000CAB2E221A5501341F2C10D80A21280063
:104C200000F0C4FB661C30310CAB19550A2128007A
:104C300000F0BCFB051E01D03400EDE73400032377
:104C4000229A1340012B1CD01F2C06D84346002B60
:104C500032D00CAB2D221A550134229B0393219B99
:104C6000029301940CAB00934B465A460799069861
:104C7000FFF7E2FA15B0F0BCBB46B246A946A04623
:104C8000F0BD219B002B13D04346002B02D10C33E7
:104C900013420FD0219B013B2193190003E00CAB81
:104CA00030221A5501348C42CED21F2CF7D9CBE7D3
:104CB0002199F8E72199F6E7229B5B0704D50CAB15
:104CC0002B221A550134C8E7229B1B07C5D50CAB14
:104CD00020221A550134C0E7FFFFEFFFFFFFEF7FEF
:104CE00065CDCD4165CDCDC1B89F0010BC9F0010F2
:104CF000B09F0010AC9F0010A8A100100000E03F82
:104D0000F0B5DE4657464E464546E0B593B082467E
:104D10008B4690461193002900D1EBE200275546BF
:104D2000119B1878002800D1E7E2252809D07C1CC7
:104D300043463A005946A847119B01331193270077
:104D4000EEE7013311930024119A11780B00203BF8
:104D5000D8B2102803D88300D048C3589F460B0010
:104D6000303BDBB2092B2CD92A292FD000230A9300
:104D7000119B1A782E2A39D000239A46119A13785B
:104D8000683BD9B2122976D88B00C549CB589F46CB
:104D900001231C4301321192D6E702231C43013246
:104DA0001192D1E704231C4301321192CCE708236E
:104DB0001C4301321192C7E710231C4301321192A8
:104DC000C2E711A8FFF726FA0A90D1E71C9B1A1D2B
:104DD0001C921868002804DB0A90119B0133119380
:104DE000C6E702231C4343420A93F6E78022D2001F
:104DF00014435A1C11925A781300303BDBB2092B32
:104E000004D92A2A07D000239A46B7E711A8FFF74A
:104E100001FA8246B2E71C9B1A1D1C9218680028F2
:104E200004DB8246119B01331193A7E70020F8E7CA
:104E300080235B002343511C119152786C2A01D0CE
:104E40001C0018E0C0239B001C430131119112E0AB
:104E500080232343511C11915278682A01D01C00F1
:104E600009E0C0231C430131119104E080235B0061
:104E70001C4301321192119B18780300253BDAB2D2
:104E8000532A00D92CE29300864AD3589F468023A8
:104E90009B001C4301321192EDE780235B001C4311
:104EA00001321192E7E7782809D0582838D06F28C6
:104EB00038D0622838D010239C430A2600E0102600
:104EC000582833D0692803D0642801D00C22944399
:104ED000630501D50122944369282AD0642828D08B
:104EE000A30500D59FE0E30500D5B8E0630600D434
:104EF000CAE01C9A111D1C911168FF220A400594FA
:104F00000A9B049353460393029600230193009255
:104F100043463A0059462800FFF76EFA070027E09B
:104F20001026CDE70826CBE70226C9E72022144346
:104F3000C8E7A30520D4E30550D4630666D51C9AC0
:104F4000111D1C911168FF220A40D317D118594036
:104F500005940A9B0493534603930296D20F019241
:104F6000009143463A0059462800FFF745FA0700EA
:104F7000119B01331193D3E61C9BDA1D07218A4351
:104F8000110008311C91116853689C46DB170C9383
:104F90000D930C9A0D9B100048400E9062465340B2
:104FA0000F930E980F990C9A0D9B801A99410E90B1
:104FB0000F9108940A9B0793534606930496002387
:104FC00005936346DA0F02920090019143463A003E
:104FD00059462800FFF76EFA0700C9E71C9A111D11
:104FE0001C911268D317D118594005940A9B049359
:104FF000534603930296D20F0192009143463A0022
:1050000059462800FFF7F8F90700B1E7230605D550
:105010001C9A111D1C910023D25E96E71C9A111D4B
:105020001C91126891E71C9BDA1D07218A4311002D
:1050300008311C9108940A9B0793534606930496E3
:105040000023059302931368546800930194434628
:105050003A0059462800FFF72DFA070088E71C9A06
:10506000111D1C9105940A9B0493534603930296C9
:10507000002301931368009343463A0059462800E1
:10508000FFF7BAF9070073E723060DD51C9A111D27
:105090001C9112681204120C31E7C046C49F001024
:1050A00008A0001054A000101C9A111D1C91126839
:1050B00025E746281AD01C9B0733072293431A0082
:1050C00008321C9204940A9A0392524602925C6837
:1050D0001B680093019443463A0059462800FFF7A5
:1050E00065FC0700119B0133119319E620231C4333
:1050F000E1E7672801D0472802D180231B011C4328
:10510000452801D0472801D120231C431C9B07338D
:10511000072293431A0008321C9204940A9A0392BD
:10512000524602925C681B680093019443463A0021
:1051300059462800FFF730FA0700119B01331193FD
:10514000EEE502231A002240924623421FD001249A
:105150001C9B1A1D1C927A1C9146187843463A00F3
:105160005946A8475346002B16D1119B0133119382
:105170004F46D5E5561C434659462020B8472300E4
:1051800032005C1C9D42F5D83D001700E0E701238A
:105190003A002F000A9DF4E74A46A9460A9D06E018
:1051A000571C434659462020C84734003A00661C25
:1051B000A542F5D84D469146D7E71C9B1A1D1C9277
:1051C0001B6899465346002B00D1013B4E4601E037
:1051D000013613003278002A02D05A1E002BF7D174
:1051E0004B46F21A10928023DB0026001E401C4220
:1051F00003D0524501D95346109302231A0022408E
:105200000B92234205D03A0037004C46A94655463A
:1052100020E03A00109B5F46B3462E0006E0551C86
:10522000434639002020B04723002A005C1C0A991D
:105230009942F4D835005E46BB46109437004C4680
:10524000A946554606E01D000134561C4346594602
:10525000C84732002078002804D0002FF4D06B1EFD
:10526000002DF0D117004D460B9B002B03D1119B55
:105270000133119354E50A9F109B06E0561C4346E8
:1052800059462020A847230032005C1C9F42F5D8D5
:105290001700ECE721231C431C9B1A1D1C921B6862
:1052A0000093059408230493534603931023029319
:1052B0000023019343463A0059462800FFF79CF823
:1052C0000700119B013311932AE57C1C43463A00E9
:1052D00059462520A847119B0133119327001FE54C
:1052E0007C1C43463A005946A847119B0133119351
:1052F000270015E50A4B9A4610E5AA46474502D312
:1053000043465A1E00E03A00434659460020D04723
:10531000380013B0F0BCBB46B246A946A046F0BD6B
:105320000542001000B585B0029003910121009361
:1053300013004A4202A90248FFF7E2FC05B000BD93
:105340000742001001480421014B1847C004002007
:105350007553001010B5010018231B881422108803
:10536000984710BD10B5010018231B88162210881D
:10537000984710BDF0B5C64600B507000E000025E1
:105380000123984600E00135B5420AD2AC003C1931
:105390002068FFF7DFFF20600028F4D10023984643
:1053A000F1E7404680BCB846F0BD0000124A936F5A
:1053B0009B0815D29066D166002905D0FFE7FFE76C
:1053C000FFE7516F106F704704B580210906C217BF
:1053D0005140002800D0C84303F0DAFE002104BD8C
:1053E000F0B5146E556E576F166FFFF7E3FF146636
:1053F000556657671667F0BD000000D0114A936FDD
:105400009B0813D210665166002905D0FFE7FFE71D
:10541000FFE7516F106F704704B5002801D00020DE
:10542000C04303F0B5FE002104BDC046F0B5146EC4
:10543000556E576F166FFFF7E5FF14665566576791
:105440001667F0BD000000D094464E4A926F920855
:10545000624601D230E0C046F0B54A4EB56F6D08E5
:10546000FCD3346E756E776F366F00F025F8944676
:10547000444A14665566576716676246F0BDC046D3
:105480009446404A926F9208624601D258E0C04664
:10549000F0B53C4EB56F6D08FCD3346E756E776F0A
:1054A000366F00F04DF89446364A146655665767D5
:1054B00016676246F0BDC046002B24DB11D00029E0
:1054C0003EDA00B5C943404200D1013100F038F85E
:1054D000C943404200D10131DB43524200D1013384
:1054E00000BD002AEBD1002801D1002905D0002001
:1054F000C90FC90701D1C043410800B503F040FE00
:105500000022002300BD00B500290ADBDB43524224
:1055100000D1013300F014F8C943404200D10131F9
:1055200000BDC943404200D10131DB43524200D1AA
:10553000013300F005F8DB43524200D1013300BDD6
:10554000002923D1002B18D1002A0CD0BC460D4FC6
:1055500038667A6600210023FFE7FFE7FFE77A6FEE
:10556000386F67467047002801D00748010000B532
:1055700003F006FE0022002300BD02000B00002005
:1055800000217047000000D0FFFFFFFF002B00D07C
:10559000BFE0130C28D1002AE7D080B4114F396640
:1055A0007A66FFE7FFE730B4040C7B6F396F1B04AA
:1055B00023433B667A66FFE7FFE7FFE7C04684B216
:1055C0007B6F3D6F1B0423433B667A66FFE7FFE773
:1055D000C04600232C042D0C7A6F386F00196941E6
:1055E000B0BC7047000000D0F0B594460025140E02
:1055F00001D112020835140F01D112010435940FA4
:1056000001D192000235D40F01D152000135D40BE3
:105610000134254F7C66254C3C660E0C93B2FFE7A7
:10562000FFE7FFE73C6F6643360C7703BE467343E4
:10563000DF0B5B04C01AB941130C7343DB18C91AA2
:10564000CE086643360CB64493B273431F0F1B015A
:10565000C01AB941130C73431F0B1B05C01AB94183
:10566000860D8F023E436643360C092D24DB520A19
:105670007243801A7703460A6643360C16235B1B77
:10568000DE40DF40BF1964466643821B7046043526
:1056900006330100D940A840C01900D30131A2420D
:1056A00006D20023F0BD0000000000D0FFFFFFFF86
:1056B000121B0130F3D3F1E709277F1BFE4064463C
:1056C000A2B27243801A00D20139220C7243130C29
:1056D0001204821A99410B007046043513370100F9
:1056E000F940A840801900D30131002B02D1A24219
:1056F0000AD2F0BD013000D30131121BFAD2013BB6
:10570000F8D1A24200D2F0BD013000D30131121B0A
:10571000F7E7F0B51C0C00D080E00CB400251C0AA3
:1057200004D11B02160E3343120208351C0B04D1A0
:105730001B01160F3343120104359C0B04D19B004F
:10574000960F334392000235DC0B02D192185B4175
:1057500001351C00971864410134464F7C66464C65
:105760003C660E0CFFE7FFE7FFE7C0463C6F664371
:10577000360C7703BE4697B27743C01B00D201397F
:10578000C01B00D201399FB27743C91BC91B170C3C
:1057900077437E04FF0B801BB941CE086643360C6D
:1057A0000C2D33DBB644120B1F053A431B0B97B28B
:1057B0007743C01B00D201399FB27743C91B170C36
:1057C00077433E043F0C801BB941860D8F023E4358
:1057D000664329277F1BFE400C3D7746AF40BF192B
:1057E00030BCA2B2ABB272437343801A9941220C0F
:1057F0007243130C1204801A994102000B00013706
:10580000001BA941F9D2781E0021F0BD0C277F1B97
:10581000FE4077467F0BAF40FF19E0E700245D1C98
:1058200007D0144F7D663966FFE7FFE7FFE7FFE724
:105830003C6F95B29EB265436643401BB141150C67
:105840001E0C6543664336042F0C3E432D04401B5B
:10585000B141994204D202000B0020000021F0BDAA
:1058600001D19042F7D3801A994101349942F2D381
:10587000F6E70000000000D0FFFFFFFF4840414076
:10588000484018B4134B5B68019308BD18B4114B22
:105890001B68019308BD94460F4A926F920805D287
:1058A000624618B40B4BDB68019308BD0A4AF0B599
:1058B000146E556E576F166F6246FFF7F2FF064A79
:1058C0001466556657671667F0BD18B4014B9B68A0
:1058D000019308BD508C0220000000D0FFB550405D
:1058E0004240504059404B40594000E0FFB5154FF1
:1058F0004C00640D03D0BC4204D10C0314D800202A
:10590000090D09055C00640D03D0BC4204D11C03E1
:105910000AD800221B0D1B0501264B4009D44B4021
:1059200003D58B4200D18242FFBD9942FCD1904207
:10593000FFBD0B43DB1803431343F5D0C94349189C
:10594000FFBD0000FF07000000B5FFF7CFFF80415B
:1059500000BDC04600B5FFF7C9FF01D9002000BD5A
:10596000012000BD00B5FFF7B9FF01D9002000BD3F
:10597000012000BD00B5FFF7B1FF804100BD01204F
:1059800040054A00121804D85A00121801D8002005
:105990007047012070470020704700000021002858
:1059A00005D17047C1174840401AFAD0C90713B54E
:1059B000064B1B6898470CBC441CA2401005120BF8
:1059C0000349091B09051943114310BD508D0220DD
:1059D0001F04000010B54C00620D8023D218DB00BC
:1059E000D21A5B057E2A10DD9E3A13DACC17090322
:1059F000490819435242D140640001341532202A2B
:105A000005DAD0400843604310BD002010BD0846B1
:105A1000604310BDC80FC018013810BD18B4024B48
:105A20005B6A019308BD0000508C022010B501484C
:105A3000FEF7A2F9F8A1001070B513231C78012C11
:105A400014D0012C14DC022C02DC1F4A1F4B9A6478
:105A50001F48FFF77FFC1F4B186070BD99001E4860
:105A60001A4A885001331F2BF8D9EAE70023FAE7D6
:105A70001A48FFF777FC05001948FFF773FC023856
:105A800003789B007F2B19DD802229000F4800F04E
:105A900017F9022CD7D1134B1A88B5231B029A424F
:105AA00009D1114B1A88114B9A4204D1104B1A8814
:105AB000104B9A42C7D00020FEF75EF90E4B0F4AFA
:105AC00032210F48FEF7BEF8055B0010508C022013
:105AD0004C330000508D02202D5A0010534400001A
:105AE0005346000054380000D838000049460000F2
:105AF0009C3800005946000010A20010B8A2001007
:105B000070A2001007B56046002800D100BE0188D1
:105B10000A0A0230DF2AFAD1C9B2820804D3028805
:105B200040880004104300E00068024A505003908F
:105B300007BD0000508C022051434343C9188C46D6
:105B4000110C83B24B4310B4040C614392B280B287
:105B5000504362431C041B0C001910BC5941130430
:105B6000120CC01851416144704700004840414048
:105B700048400E4B5B6818470C4B1B6818470C4A93
:105B8000936F9B0802D2094BDB681847F0B5146E7F
:105B9000556E576F166FFFF7F6FF054A1466556688
:105BA00057671667F0BD014B9B681847548D02205C
:105BB000000000D0491A002808D1084670470000AC
:105BC000C10FC90700D54042002817D0F44603B4DE
:105BD0000B4B1B68984706BC81409E384042803181
:105BE00007D20B0607D04900490AC00510430843F5
:105BF00060470130F8E7490A8902F5E7704700007D
:105C0000508D0220014B5B6A18470000548D022022
:105C100010B50148FEF7B0F8BC92001070B5132320
:105C20001E781848FFF79EFB0500012E11D0012EAB
:105C300009DDAB1E1B789B007F2B1DDD8022290018
:105C4000114800F03DF81148FFF784FB104B186035
:105C500070BD542201000C4800F032F8002300E02F
:105C600001331F2BE3D89A00074C1259002AF7D1B1
:105C70009A0008481051F3E7074B084A42210848A8
:105C8000FDF7E0FF53460000548D02204C33000026
:105C9000508D0220115C0010CCA2001044A3001013
:105CA00000A3001001480421014B1847D004002034
:105CB00075530010014B1B6818470000D0040020EA
:105CC000014B5B6818470000D004002010B50300AA
:105CD000080011001B68984710BD0000F8B50700C8
:105CE0000D001600437C002B02D0002400200CE0A5
:105CF00003681100280098472DE03B7C10E002214A
:105D000015483B689847601C0134B44214DA002CF3
:105D1000F3DD2B19013B1B780D3B5A425341DBB29B
:105D20002A5D0A2AF0D1002BEED1A042E7DA211A2F
:105D300028183B689847E2E7B04203DA311A28187E
:105D40003B689847002E06DDAD19013D2B780D3BD1
:105D50005A4253413B74F8BD44A4001070B505008D
:105D60000368002B16D00C4B1C6805E0290004C901
:105D70002000FFF7B3FFE468002C09D02368002B54
:105D8000F9D0064B1B68002BF0D0A342F3D1EDE70E
:105D900000232B6070BDC0467C87022080870220D4
:105DA00070B505000C000B68802B05D021684B1CDA
:105DB00023606418257170BD0800FFF7CFFFF5E779
:105DC000F0B583B007000E000092019328E0A368AD
:105DD000002B04D0310038009847002827DCE46805
:105DE000002C06D0134B1D68002DF0D0A542F6D133
:105DF000EDE70099019A104B5B6A9A4209D80E4868
:105E0000806A88420FD29A4201D0012302E0002327
:105E100000E00023002B08D101200021FDF7A2FBA8
:105E2000064B1C68DCE70123F4E70120404203B085
:105E3000F0BDC04680870220004005407C870220DC
:105E400010B582B0D0231B0600241C5701A90748B7
:105E500003F0A6F9002806D1019B9C4203D0034819
:105E600003F0AEF9012002B010BDC04628050020A5
:105E700010B5024803F07CF910BDC046280500208B
:105E8000F0B5CE46474680B583B006000D0090467B
:105E90001C00FFF7D5FF81466B1C05D0002C08D0F5
:105EA000194F1A4B1C6807E0300003F027F9050072
:105EB000F4E7174FF5E7E468002C17D02368002BB0
:105EC000F9D0144B1B68002B01D0A342F3D12A0058
:105ED00031002000B8474346002BECD06B46D91D5B
:105EE0000A230B7001222000B847E4E74B46002B41
:105EF00007D16B1E9D41E8B203B0C0BCB946B046A5
:105F0000F0BDFFF7B5FFF4E7CD5C00107C87022001
:105F1000DD5C00108087022010B582B004006B4663
:105F2000D81D0470012300220121FFF7A9FF2000E2
:105F300002B010BD094A01E00C331A001368002BAF
:105F400008D08342F8D1002907D1C3681360002329
:105F5000C36002E0002900D0106070477C870220F7
:105F600010B5064B1C6801E09847E468002C03D08C
:105F70006368002BF8D1F8E710BDC0467C8702208B
:105F800070B5050003F0BAF80400002301220100F7
:105F90002800FFF775FFFFF7E3FF200070BD00004A
:105FA00070B5A2B004000E00FFF74AFF050084227E
:105FB000002101A8FFF77EFE3300220001A9084856
:105FC000FFF7B0F9040001A8FFF7C8FEFFF7C8FF0C
:105FD000002D02D1200022B070BDFFF749FFF9E784
:105FE000A15D00100FB400B583B004A901C90191EF
:105FF000FFF7D6FF03B008BC04B0184710B500F097
:1060000093F910BD30B583B004000025FDF78AFA7E
:1060100002000B1E16DB12196B41994202D804D103
:10602000904202D901225242D317002B10DB0121EA
:1060300001A8FFF7C5FE002802DB0FD001AB1878DE
:1060400003B030BD094B0A4A3F210A48FDF7FAFD6B
:10605000064B074A3F210748FDF7F4FD9521064B03
:10606000064A49000648FDF7EDFDC0466498001059
:1060700018A40010809800109099001030A400100F
:10608000DCA3001070470000014B00221A7070471B
:10609000A28E02204B79FF2B0CD18B79002B0BD1D8
:1060A000CB79012B0AD1082A0AD98A78054B1A70B4
:1060B000092000E0002070470020FCE70020FAE7FC
:1060C0000020F8E7A28E02200120704770B504007E
:1060D0000D000348FFF73EF9030029002000984710
:1060E0005542000010B5002926D1117953791B02C1
:1060F0000B43124909788B4201D0002010BD537820
:10610000012B03D0022B10D00020F7E79178D37831
:106110001B021943DB0503D54B0A0120984000E020
:1061200000207F231940FFF7D1FF642200210020C7
:10613000FEF730F80120E1E70120DFE7A28E022020
:10614000012303700048704748A4001010B50B7875
:106150004878000218438A7812041043CB781B0653
:1061600003439622D200934200D010BD00210800C4
:10617000FFF7ACFF30B583B005000C0001A918484B
:1061800003F00EF8002808D1D0231B061B68019AE3
:106190009A4221D0124803F013F8002001F054FE77
:1061A000002807D1032464420D4802F0E1FF2000DB
:1061B00003B030BD002001F069FE002802D10324A5
:1061C0006442F1E722002900002001F06BFE041E6A
:1061D000EAD103246442E7E703246442E7E7C046C8
:1061E000608E022010B50021054802F0D9FF00287A
:1061F00000D110BD01F0C0FB014802F0B9FFF8E783
:10620000608E0220F0B5C64600B582B080460D0013
:1062100001A92E4802F0C4FF002808D1D0231B0694
:106220001B68019A9A420FD0284802F0C9FF00204B
:1062300001F00AFE002847D1254B002000211860FC
:106240005960224802F094FF02B080BCB846F0BD0D
:1062500001F092FB002001F039FE002001F0F4FD76
:106260000028EED0002001F0B3FE00281DD0AC4283
:10627000E7DA2E1B002001F0ABFE0200864200DCB4
:106280003200002AE4D043461919002001F084FEB0
:10629000060001F071FB002001F018FEA419FDF7C3
:1062A00041F90B4B18605960E1E7FDF73BF9084BEA
:1062B0001E685F68074A002392197B419942C0D843
:1062C000D5D19042D3D9BCE70024D0E7608E02201C
:1062D0000081022020A1070010B50A4B1A78D023B4
:1062E0001B061B689A4207D1074B1878FCF75EF82B
:1062F000FA208000002110BD044B054A32210548D8
:10630000FDF7A0FCAB8E0220AA8E022060A4001034
:1063100004A5001088A4001010B5024B1878FCF7F3
:1063200045F810BDAA8E022070B584B0D0231B069C
:106330001A782D4B1A702D4B1B7802F08FF82C48D1
:10634000FDF74AFC0120FCF7EFFAC0B2294C20709F
:106350002949FCF74DF820780121FCF71FF80520AA
:10636000FCF734F8041E0BD0002224490520FCF76A
:1063700069F801212248FFF7DDFD200004B070BD5F
:10638000FCF744FE0600FDF7CDF804000D1E1EDBF1
:106390000100FA229200002312196B419D4202D89B
:1063A00004D1914202D901225242D317002B14DBAF
:1063B0000121029100210191124900913000FCF766
:1063C0003BFE431E9841C4B20028D6D0D1E70E4B05
:1063D0000E4A3F210E48FDF735FC0B4B0B4A3F217F
:1063E0000B48FDF72FFCC046AB8E02202CAD0010F1
:1063F000608E0220AA8E0220E56100101963001051
:10640000E0040020D962001064980010ECA4001091
:10641000809800100048704790A500100048704711
:106420003CA5001010B50400154B1B78002B0ED0B6
:10643000002C11D1134B144A5A80012301335B0005
:106440001BB2C022920013430E48038010BD1121DD
:106450000B4802F0D7FBEBE7052C0ED8A4000B4B42
:10646000E4580023122BE9D8E25C002AE6D001337D
:10647000590004484252DBB2F4E70020E6E7C04688
:10648000808E02204487022009040000A4A5001089
:1064900002007F201040D209400080184001014BCB
:1064A000C01870478487022010B582B001AB074A3C
:1064B0001A80002406E001AB185DFFF7E9FF012315
:1064C000C3700134012CF6D902B010BD0080FFFF6B
:1064D00010B5838B3F333F229343022915D0124CD2
:1064E0002268C260D31823609C0610D10F4C624012
:1064F000634080246401A3420FD88906114380239E
:106500001B0619434368196010BD5B00E7E7084BA1
:10651000084A54210848FDF795FB084B054A5621C7
:106520000548FDF78FFBC046308C0220000010505C
:10653000BCA50010D4A60010ECA5001040A60010C9
:10654000F8B505000E001400FFF7A2FF7F232B40D3
:10655000EF0985707A427A4142700022C2708683C8
:106560008477012F0DD0DA0012498C466244826094
:10657000826800211160002B09D143600E4BC3607B
:10658000F8BDDA000D498C4662448260F0E7012FC5
:1065900009D0013BDB000A4A944663444360210072
:1065A000FFF796FFECE7013BDB00064A94466344A5
:1065B0004360F4E784001050000110508000105038
:1065C0000C0010500800105010B5002308E00133F3
:1065D000DA00002108481150844662445160DBB261
:1065E0000E2BF4D9F022920000210448FFF762FB41
:1065F000034B044A1A6010BD00001050C4870220EB
:10660000308C022080011050F0B5CE46474680B550
:1066100083B01D4B9F6D0024012603E0B743760035
:106620000134E4B2002F29D01F2C27D83E42F6D0E7
:10663000164B9E65630899460123634001221A4068
:1066400090464B465D0045446D01114BED18280006
:1066500000F0ACFA0028E1D04B465B0043445B01FC
:106660000B4AD3189A8A99780123009300230020BB
:1066700000F00AFE280000F009FACFE703B0C0BC22
:10668000B946B046F0BDC046000011500030115070
:106690008487022070B52B4A9823D45880235B024C
:1066A00025001D401C420AD1E30616D4E30419D488
:1066B000630429D4230433D4A5423ED170BDFFF72F
:1066C000F3FE01222049002000F0C4FD1F4B802270
:1066D00092021A6580256D02E6E710231D43FFF73D
:1066E00093FFE3E780235B011D43164B00221A60F2
:1066F000FFF76AFF01220021002000F096FD134BF6
:10670000802212031A65D3E78023DB011D43012297
:106710000421002000F076FD0C4B10221A65C9E719
:1067200080231B021D4301220521002000F06AFD89
:10673000064B802212011A65BEE729006140044819
:10674000FDF71AFB000011500000105000301150EE
:1067500074A6001070B50C001500FFF799FE2A0012
:10676000210000F0FFF970BD10B5002804D101210F
:106770000520FBF713FE10BDB921034B034A490066
:106780000348FDF75FFAC04688A60010C4A60010B3
:10679000ECA5001010B5002805D1002200218020B2
:1067A000FFF7D8FF10BDBF21024B034A4900034841
:1067B000FDF748FA88A60010B4A60010ECA500105A
:1067C000024B80225202DA647047C046002011500A
:1067D00070B5041E25D100F033F9154D0C23AB67BD
:1067E00014490520FBF704FE402200211248FFF760
:1067F00061FA002240210020FFF7A2FE0022402182
:106800008020FFF79DFEFFF7DFFE01232B6480232E
:106810009B05EB649023094AEA502000FFF7D0FF64
:1068200070BD4E21064B074AFF310748FDF70AFAB3
:1068300000001150956600108487022010D00100DE
:1068400088A60010E8A60010ECA500100B785B06E7
:1068500002D14B78052B00D070478A78014B1A6023
:10686000FAE7C0460000115010B50C0000280DD109
:106870000A794B790721194009021143E2789207FE
:10688000920FA078FFF75CFE012010BDD621034BCC
:10689000034A49000348FDF7D5F9C04688A6001011
:1068A000A4A60010ECA5001010B5FFF78DFE10BDDA
:1068B00010B50400080011001A00002C03D1FFF7E6
:1068C00049FF012010BDBC21024B034AFF310348A0
:1068D000FDF7B8F988A6001094A60010ECA50010EA
:1068E00010B508004B0605D1CB09012B0AD00222B6
:1068F000054B9A66FFF7CCFD80221201002100F0C3
:10690000CBF810BD0122F3E70020115010B50800AC
:106910004B0600D110BDFFF7BBFD0023C370002262
:10692000014900F0B9F8F5E7FFF7FFFFF8B50400FB
:106930000F00438A828B1E1C934200D9161CB6B2EC
:106940009B1B63828025ED003543E378002B13D039
:1069500080229201154301225340E3706378002B9B
:106960000CD0638A002B02D18023DB011D43002F52
:1069700000D02D042800F8BD0022EBE7B801E36841
:106980009C4660443200A169FFF79AF9A3699C46CE
:106990006644A66180231B021D43E2E770B5040034
:1069A00083681B68002900D01B0C9D05AD0D627823
:1069B000002A11D11B0409D4A38A5B19A382A38BDB
:1069C000AB4201D900236382280070BD0E4B0F4AF1
:1069D000D7210F48FDF736F91B040ED58901E3686E
:1069E0009C4661442A00A069FFF76AF9A38A5B19F3
:1069F000A382A3695B19A361E1E7064B034ADE2189
:106A00000348FDF71FF9C046F4A6001014A80010B3
:106A100014A7001068A7001010B5040083681B6855
:106A20000021FFF7BBFF63681B685B0002D5A38BE7
:106A3000834200D010BD01212000FFF7AFFFF9E72E
:106A400010B580235B040C4A13600C4A13600C4B96
:106A50009A6880235B049343F9D10A4C9C2200215D
:106A60002000FFF727F98022520100210648FFF796
:106A700021F90923636710BD00E0004000F00040E9
:106A800000C00040000011500000105000230374AB
:106A9000438283828361704710B5002902D08368E6
:106AA0001B681940002A0FD0114353050CD582688A
:106AB00013685B050BD40B4B0B401360FFE7FFE73C
:106AC000FFE7FFE7FFE7FFE78368196010BD837802
:106AD0007F211940DB099B00034A9A580348FDF7C0
:106AE0004BF9C046FFFBFFFFF404002088A700100D
:106AF00070B5040043681E680021FFF717FF80256A
:106B00006D010543144B1B6C9B0704D4A378DB0970
:106B100014D1013300E00023628A002A01D0002B47
:106B20000ED00E4B1E4080239B05334362681360DA
:106B30002A0000212000FFF7AFFF70BD0023EBE724
:106B400001212000FFF7F2FE0543054B1E40A02364
:106B5000DB053343EAE7C04600001150FFFFFFAFFB
:106B6000FFFFFFDF70B504000D001600037C002B53
:106B700009D166820023A38201332374A56120001A
:106B8000FFF7B6FF70BD83787F211940DB099B00BA
:106B9000044A9A580448FFF725FA2000FFF776FFC9
:106BA000E7E7C046F4040020A8A7001070B5040071
:106BB000057C002D06D0FFF72FFF638A002B08D13C
:106BC000280070BD81787F231940044A0448FDF7EE
:106BD000D3F82000FFF78CFF0025F1E7F404002034
:106BE000E0A7001070B5050000240EE063001B193B
:106BF000DA00184B1B689B1802E0230010E000230A
:106C00005B68280098470134E4B2134B1B78A34219
:106C10000ED3124A002AF0D0A342E7D8E31ADBB21F
:106C2000002BECD15A00D218D2000D4B9B18E7E78D
:106C30000C4C532200212000FFF73CF8E01C1022EE
:106C4000FF21FFF737F8200013302022FF21FFF744
:106C500031F870BD64810220988E022041610010DD
:106C60005CA900109C84022010B5FFF7BBFF01F067
:106C70002BF810BD70B505000C001600C86801F0B7
:106C80002DF8E368320000212800984770BD00000D
:106C9000F0B5DE4657464E464546E0B583B08146E0
:106CA0000139C8B2FFF7BAFB002803D043789846F1
:106CB000022B0CD0564A57495748FFF793F900204A
:106CC00003B0F0BCBB46B246A946A046F0BDC579AC
:106CD0006A11012351491A4014010A781026B2435F
:106CE00022430A70AD112B405B01D2B22024A24393
:106CF00013430B70070009378178C3781B020B43DD
:106D000082469A4463E0FB789B463B78FF1865E037
:106D1000434A40494048FFF765F90020D0E7660044
:106D20003619F3003F4A1668F61802E0230017E010
:106D300000262A0039004846B36898470190082881
:106D400001D9854214D20134E4B2374B1B78A342F7
:106D500039D3364A002AE9D0A342E0D8E31ADBB29D
:106D6000002BE5D15E00F318DB00314EF618E0E7AA
:106D70005B46012B10D0002293451AD9BB789B1893
:106D8000DBB22649C918C978FF290BD12349CB1892
:106D9000DC700132D2B2EFE7B268264B9A42EAD1F8
:106DA000C346E8E7244A1B491B48FFF71BF90020AC
:106DB00086E71A482300019D2A003900133001F0AC
:106DC000BBFBAC466744184B1B78A3420ED3574518
:106DD00014D27B780B2B96D001239B467B78042B17
:106DE00096D15346DD1BADB20024AEE7F3229200EC
:106DF00008490948FFF7F6F8002061E70F4B002B20
:106E000003D000E000BF01205AE7012058E7C04648
:106E10007B03000024A9001024A800109C840220F9
:106E20009603000064810220988E022041610010C8
:106E30005CA90010ED800010BD0300000000000000
:106E400070B505000C00CB7888780F2B54D89A00C9
:106E50002F498A589746FFF7DDFA020012232100D6
:106E6000280000F0DDFE48E02A4B002B46D000E071
:106E700000BF02008178C3781B020B432100280069
:106E800000F0CEFE39E0022B10D0234B002B37D080
:106E900000E000BF0200002A0CD09178D3781B02DA
:106EA0000B432100280000F0BBFE26E0FFF7B6FAF6
:106EB0000200F0E7194A1A491A48FFF793F8002030
:106EC0001BE02379617909021943FFF7ABFA021E2F
:106ED00018D003782100280000F0A2FE0DE0124B2C
:106EE000002B11D000E000BF021E0FD0037821005C
:106EF000280000F095FE00E0002070BD0020FCE7B7
:106F00000020FAE70020F8E70020F6E70020F4E789
:106F10003CA8001000000000000000001404000065
:106F20000CA9001024A8001000000000024B5878A3
:106F3000431E9841C0B270479C840220024B1878CF
:106F40004007C00F7047C0469C840220014B187850
:106F50007047C046998E022070B50500274B1878FF
:106F6000002800D070BD532200212548FEF7A2FE64
:106F7000244C2000FCF730FE234B1C60234C2000E7
:106F80001C30FCF74FFE200001F0F0FD204B1C6090
:106F9000204B002B04D02048FFF7D2F81F4B18607D
:106FA00000240DE063001B19DA001C4B1B689B18C2
:106FB00002E023000FE000231B6898470134E4B28D
:106FC000154B1B78A3420ED3124A002AF1D0A342DC
:106FD000E8D8E31ADBB2002BEDD15A00D218D20068
:106FE0000F4B9B18E8E72800FFF7F2FB2800FFF79C
:106FF000BBFB024B01221A700120B3E7998E0220DD
:107000009C84022054840220F0840220FC0400208E
:10701000F484022041610010988E022064810220D5
:107020005CA9001030B585B004004378042B00D172
:1070300096E038D8022B62D0032B00D0B9E06D4B1C
:107040001B785B0700D483E06A4A137804218B43E2
:1070500013700C22002101A8FEF72CFE23786A464B
:10706000137105235371644B1C68E269EFF31081BF
:1070700072B61368002BFCD0BFF35F8F216201A9A9
:10708000200001F038FDE269236ABFF35F8F002121
:10709000116083F3108800285AD1A8225749584814
:1070A000FEF7A0FF54E0052B00D082E0514B1B7887
:1070B000DB074DD54F4A137804218B4313704E4B99
:1070C0001D68EA69EFF3108172B61368002BFCD0DB
:1070D000BFF35F8F29622100280001F00CFDEA69EF
:1070E0002B6ABFF35F8F0021116083F310880028A3
:1070F0002ED1A82241494248FEF774FF28E03D4BBB
:107100001A7801218A431A701A7801318A431A7059
:1071100000225A701A7802318A431A70364B1D6861
:10712000EA69EFF3108172B61368002BFCD0BFF34D
:107130005F8F29622100280001F0DDFCEA692B6ADB
:10714000BFF35F8F0021116083F31088002801D006
:1071500005B030BDA82229492948FEF743FFF7E7CB
:10716000244B1B78DB07F3D5224A137804210B4309
:107170001370214B1D68EA69EFF3108172B6136832
:10718000002BFCD0BFF35F8F29622100280001F0A3
:10719000B2FCEA692B6ABFF35F8F0021116083F3B1
:1071A00010880028D4D1A82214491548FEF71AFFE8
:1071B000CEE7114B1D68EA69EFF3108172B61368D0
:1071C000002BFCD0BFF35F8F29622100280001F063
:1071D00092FCEA692B6ABFF35F8F0021116083F391
:1071E00010880028B4D1A82204490548FEF7FAFE09
:1071F000AEE7C0469C840220F4840220FCA8001064
:1072000024A8001070B584B006000D0014000C22F4
:10721000002101A8FEF74EFD6B461E715D71210035
:1072200001A8FFF7FFFE04B070BDF0B585B0070000
:107230000E00150001AC0C2200212000FEF73AFDE3
:10724000277001236370267129002000FFF7EAFEF2
:1072500005B0F0BD70B584B006000D0014000C221E
:10726000002101A8FEF726FD6B461E7106236A4623
:1072700053710822290002A8FEF722FD210001A86F
:10728000FFF7D0FE04B070BDF0B5CE46474680B5DE
:1072900085B080460F0016001D000CAB1B78994688
:1072A00001AC0C2200212000FEF704FD43462370B0
:1072B0000723637027710396657149462000FFF725
:1072C000B1FE05B0C0BCB946B046F0BD70B5060011
:1072D0000D008B7870221A420DD10D4B9978280041
:1072E00001F0D6F8041E0DD029003000FFF7BCFADB
:1072F0000400200070BD074A07490848FEF772FEE7
:107300000024F6E7064A04490448FEF76BFEF0E75E
:107310009C840220C2040000D8A8001024A80010F9
:10732000C3040000F0B5D6464F464646C0B5814678
:107330000C0017009846089B9A46002516E0184A4C
:1073400018491948FEF74EFE00263000E0BCBA4648
:10735000B146A846F0BD154A12491348FEF742FE51
:10736000F3E7099A13702378E4180135AF4214DD6E
:107370006378052BE3D1E1788907890F4145DED198
:1073800021004846FFF7A2FF061EE4D0A378DA09E1
:10739000012AE6D052461370E5E70126D5E7C0463C
:1073A0009C040000E8A8001024A800109D04000020
:1073B00070B57F250D40CC096A001E4B9B181B1928
:1073C0003033DB78DB07DE0F002B30D1194B9B18F5
:1073D0001B193033DB785B072AD4174B186801215F
:1073E000494201F0E5FE6A00124B9B181B1930332D
:1073F000DB78DB0708D40F4B9B181B193033DB7885
:107400005B0712D5002600E00026002E08D06D0094
:1074100008494D192C193034E37804221343E370E2
:10742000054B186801F0A4FE02E00126EDE70026F6
:10743000300070BD9C840220F084022070B57F254E
:107440000D40CC09154B18680121494201F0B0FEEE
:107450006A00134B9B181B193033DB78DB0708D409
:107460000F4B9B181B193033DB785B0713D40026B6
:1074700000E00026002E08D06900094D6D182C1977
:107480003034E37804229343E370044B186801F02E
:107490006FFE300070BD0126ECE7C046F08402208C
:1074A0009C840220F0B5C64600B582B001937F25CA
:1074B0000D40CE096F00174CE419A4193034E4785C
:1074C000E4071DD46F00134CE419A4193034E37899
:1074D0000127BC4667463B43E370019BFFF7E8F991
:1074E000002813D16D000B4B5D19AE193036F378BF
:1074F00001229343F370F37803329343F37005E072
:10750000054A06490648FEF76DFD002002B080BC22
:10751000B846F0BD9C8402200A050000C8A80010EF
:1075200024A8001070B57F240C40CD0962000C4BDC
:107530009B185B193033DB789B0700D570BDFFF7D4
:10754000CFF96300064CE41864193034E378022262
:107550001343E370E37801221343E370EEE7C04680
:107560009C84022070B57F240C40CD0962000C4B36
:107570009B185B193033DB789B0700D470BDFFF795
:10758000C5F96300064CE41864193034E37802222C
:107590009343E370E378013A9343E370EEE7C04628
:1075A0009C8402207F220A40CB095200034989189B
:1075B000C9183031C8788007C00F70479C840220FA
:1075C000F0B5C64600B582B005000C00002000F002
:1075D00085FB237860221340602B12D0402B17D0FC
:1075E0002278D206D20E012A00D1D9E0022A00D197
:1075F00020E1002A1AD00026300002B080BCB84634
:10760000F0BDCC4ACC49CD48FEF7ECFC0026F3E7B0
:10761000CB4B002B00D181E1180000F05FFB220072
:107620000021280000E000BF0600E5E7202B0AD07B
:10763000002B00D07AE16378092B00D978E19B0018
:10764000C04AD3589F4623790F2B00D968E1BE4A20
:10765000D318DB78BD4A002A05D0BD4A1278934280
:1076600012D39B1ADBB2002B00D05BE15900CB1880
:10767000DB00B849C918002900D155E122002800D3
:10768000FFF7F8FA0600B7E75900CB18DB00B24A5B
:107690001168C918EFE7200000F026FBA178280048
:1076A000FFF778F8A84A137802210B4313700126DC
:1076B000A2E7A54B5B786A460632137001232100CE
:1076C000280000F0ADFA012696E7A7789E4B5B787C
:1076D000DBB2BB4205D09C4B5B78002B09D1002F5D
:1076E00013D1994B5F702100280000F07DFA01262C
:1076F00082E72800FFF7D8F8934EB3789846280021
:10770000FFF770FA4346B370E9E739002800FFF746
:10771000BFFA061EE5D1914A87498848FEF762FC08
:107720006AE721002800FFF78BFB060064E7A278D8
:10773000E3781B021343012B01D000265CE7824A49
:10774000137808210B4313702100280000F04CFA35
:10775000012651E7A278E3781B021343012B01D0E5
:10776000002649E7784A137808218B4313702100DB
:10777000280000F039FA01263EE7734B1A785109C8
:10778000920801230B4002210A4013436A46063245
:10779000138002232100280000F042FA01262BE783
:1077A00023790F2B00D9DDE0674AD318D978674BCE
:1077B000002B05D0664B1B78994229D3C91AC9B250
:1077C000002900D0D0E04B005B18DB006149C918EC
:1077D000002900D1CAE022002800FFF74BFA061E5C
:1077E00000D009E7237860221A4200D004E76378CA
:1077F0000A3B012B00D9FFE6002000F06FFA637806
:107800000A2B0CD02100280000F0EEF90126F3E647
:107810004B005B18DB00504A1168C918D8E76B466B
:107820009A1D0023137001332100280000F0F8F99D
:107830000136E1E621797F220A40CE097020084214
:1078400020D15200404882189219D27C3F4800282B
:1078500005D03F48007882421BD3121AD2B2002AC8
:107860001ED15600B218D2003A4EB618002B19D0CD
:10787000002E00D17CE0220031002800FFF7FAF949
:107880000600B9E6364A2C492C48FEF7ABFB002629
:10789000B2E65600B218D2002F480668B618E5E7DF
:1078A0000026E3E76378012B12D0032B10D0002BC6
:1078B00001D00026A0E62800FFF774FE6B469A1D53
:1078C000108002232100280000F0AAF9012693E687
:1078D000A778E27812023A4304D1012B1AD028008B
:1078E000FFF720FE002E45D0220031002800FFF7D0
:1078F000C1F9002000F0F2F9134A3423D35CDB070E
:10790000DE0F002B00D077E62100280000F06CF994
:10791000012671E62800FFF725FEE3E700266BE667
:10792000002669E6002667E6002665E6002663E68F
:10793000002661E67F02000038A9001024A800108C
:10794000000000007CA800109C840220416100100F
:10795000988E02205CA9001064810220D3020000EE
:1079600033030000002647E6002645E6002643E6EE
:10797000002641E601263FE630B585B000F080FDE7
:10798000002808D105B030BD01AC2078FFF76CF9B4
:107990002279724B9A70724B1C68E269EFF3108186
:1079A00072B61368002BFCD0BFF35F8F216201A970
:1079B000200001F07AF8E269236ABFF35F8F0021AB
:1079C000116083F310880028DCD001AB5B78082BB2
:1079D000E1D89B00634AD3589F4601AB1878FFF764
:1079E00043F9614B002BD6D000E000BFD3E75B4BDF
:1079F0001A78012401210A431A703322995CA143A9
:107A00009954995C0420814399540132995CA143B3
:107A10009954995C8143995401AB187802A9FFF7F6
:107A2000CFFD0028B7D101AC20780021FEF758FF28
:107A300020788021FEF754FFADE701AB19797F2252
:107A40000A40CC095000454B1B181B193033D8781D
:107A50000125A843D870D8780335A843D870002AE8
:107A60001DD052003D4B9A181219D37C3F4A002A70
:107A700005D03F4A1278934218D39B1ADBB2002BF1
:107A80001BD15A00D218D2003A4B9B18002B14D0AD
:107A90001C6901A84279039B0078A0477BE701A8F5
:107AA0004279039B007800F02DF974E75A00D21850
:107AB000D200314B1B689B18E8E7304A3049314807
:107AC000FEF790FA5EE7254B1B78DB0700D462E7F0
:107AD0002D4B002B00D15EE7204B18780007C00F1C
:107AE00000E000BF57E71D4B1B78DB0700D452E7CF
:107AF000264B002B00D14EE700E000BF4BE76300B0
:107B00001B19DA001C4B1B689B1802E0230014E0D1
:107B100000235B69002B02D001AA1078984701343A
:107B2000E4B2134B1B78A34200D234E70F4A002A79
:107B3000ECD0A342E3D8E31ADBB2002BE8D15A0021
:107B4000D218D2000B4B9B18E3E70024E9E7029B15
:107B5000002B00D11FE7039898471CE79C84022064
:107B6000F4840220A4A8001000000000416100106D
:107B7000988E02205CA90010648102203702000068
:107B800050A9001024A80010000000000000000010
:107B9000F8B50500124B9F89DE89B91B89B20B1C11
:107BA000402900D940239CB20D4B1B785BB2002BBF
:107BB00008DB0021B74211D00A4A23002800FFF752
:107BC00071FCF8BDB74201D18021F3E7044B9968FD
:107BD00022000448FEF774F88021EBE70022ECE76E
:107BE000408402205C84022070B506000C000B4D1E
:107BF00008222800FEF764F80023AB60EB81AB811C
:107C00000023E356002B06DB8021002300223000F6
:107C1000FFF748FC70BD0021F7E7C0464084022012
:107C2000F0B5C64600B580460C0016001D00234F77
:107C300008223800FEF744F8BE600023FB81A379D8
:107C4000E179090219430B1CA94200D92B1C99B2F6
:107C50001A4A9381A279E3791B02134319D00029B0
:107C600001D0002E08D04046FFF792FF041E0AD034
:107C7000200080BCB846F0BD732211491148FEF7C0
:107C8000B1F90024F4E779220D490E48FEF7AAF96C
:107C9000EEE70023E356002B0DDB802100230022BA
:107CA0004046FFF7FFFB041EE2D17E22044905484F
:107CB000FEF798F9DCE70021F0E7C0464084022097
:107CC0008CA9001024A8001010B51422002102482D
:107CD000FDF7F0FF10BDC04640840220014B186143
:107CE0007047C0464084022010B50100044C0822B1
:107CF0002000FDF7E5FF0023A360E381A38110BD11
:107D00004084022070B505001C00C909374B1B7860
:107D1000DB098B4219D0002C10D1354B002B02D03F
:107D20003249FEF793FD314B1B69002B03D02F4ADC
:107D30000221280098470124200070BDAB222D4964
:107D40002D48FEF74FF90024F6E7284B1B785BB26D
:107D5000002B07DB254B9868002844D022002749D8
:107D6000FDF7AEFF214AD3891B199BB2D3819168DD
:107D700009199160D288934201D03F2C28D81B4B1F
:107D80001B69002B05D0194A0121280098470028BB
:107D900014D0164B1B785BB2002B0DDB8021002327
:107DA00000222800FFF77EFB041EC5D1D82211490E
:107DB0001148FEF717F9BFE70021F0E7002128007E
:107DC000FEF78EFD80212800FEF78AFD0124B3E72F
:107DD0002800FFF7DDFE041EAED1E3220549064868
:107DE000FEF700F9A8E70024A6E7C0464084022079
:107DF0004D68001074A9001024A800105C840220B3
:107E000070B5040005001035280000F03EFE3F2844
:107E100000D870BDE1780020FFF7CAFA0028F8D03A
:107E2000280000F032FE3F2808D996239B00E21874
:107E3000E17840230020FFF735FBEAE7E1780020F6
:107E4000FFF7FCFAE5E7000010B50400FFF76EF855
:107E500000280CD10022002A11D0B6239B006343D6
:107E60000948C0180379DB070BD5012008E0FFF7AC
:107E700065F8002801D10122EDE70022EBE70020A0
:107E800010BD0020FCE7C0466881022010B5B62373
:107E90009B0058431030024BC01800F0DBFD10BDB2
:107EA0006881022070B5B6239B005843064BC51865
:107EB00092B21030C01800F019FE04002800FFF73D
:107EC0009FFF200070BDC0466881022070B505008C
:107ED000FFF72CF8002804D10023002B09D1002043
:107EE00070BDFFF72BF8002801D10123F5E700232F
:107EF000F3E7B624A4006C432834244BE41804347C
:107F0000200000F0A7FD002801D10020E8E7B622FC
:107F100092006A431D4B9B1899780020FFF748FA9E
:107F2000002801D10020DBE7B626B6006E43A62369
:107F30009B009C466644154BF618402231002000F9
:107F400000F0D4FD041E15D0B620800068430F4D0C
:107F50002D18A978230032000020FFF7A3FA00288B
:107F600001D02000BCE7C82209490A48FEF73AF8C8
:107F70000020B5E7B62080006843044D2D18A9788D
:107F80000020FFF75BFA0020AAE7C04668810220C4
:107F9000BCA9001024A8001070B50500B624A400E8
:107FA00044432834094BE418043492B2200000F012
:107FB000D8FD0600200000F04DFD3F2801D830001C
:107FC00070BD2800FFF782FFF9E7C04668810220F4
:107FD00010B5B6239B0058432830034BC01804301B
:107FE00000F053FD10BDC04668810220F0B5CE46BA
:107FF000474680B583B0B622920000212848FDF79D
:1080000059FE0026002E04D003B0C0BCB946B046CD
:10801000F0BD234FB624A40074433D19FF236B71B8
:10802000002398461F4AEA8001222A81AB72EB7234
:1080300008232B7321004831C919F83399462000D1
:108040001030C0194346009301334A4600F0C9FC82
:1080500021004931FF31C91920002830C0190430EE
:10806000012300934A4600F0BCFC92239B00E318D6
:108070009946B9444846FBF7AFFD43466B624B4611
:10808000AB6294239B009C466444E4192000FBF7F8
:10809000A3FD2C6443466B640136F6B2B2E7C046DA
:1080A0006881022000C2FFFF70B50025002D00D0BE
:1080B00070BDB624A4006C430B4EA019052200210C
:1080C000FDF7F8FD20001030801900F04FFD283436
:1080D000A4190434200000F049FD0121200000F023
:1080E0006BFD0135EDB2E1E768810220F0B583B0A8
:1080F00006004B79022B68D18B79022B69D10023C2
:10810000002B08D00027002F13D08B783B700C7801
:108110000C19092519E0B624A4005C432E48001967
:108120008078002802D00133DBB2E9E72A4FE71953
:10813000E9E78F22520029492948FDF753FF00251E
:1081400044E021784D19ADB264186378242B01D135
:108150009542F6D9052B09D06378042B02D16379B7
:108160000A2B18D03800FFF74BFE2FE0210030001B
:10817000FFF7ACF8002806D0A3787B702278551959
:10818000ADB2A418E8E79922520014491448FDF74B
:1081900029FF00251AE021784D19ADB26118BB1CEA
:1081A0000193FB1C0093022302223000FFF7BAF870
:1081B000002802D00E35ADB2D4E7A1225200074903
:1081C0000748FDF70FFF002500E00025280003B059
:1081D000F0BD0025FAE7C04668810220B0A9001072
:1081E00024A80010F8B51400127860231340202B47
:1081F00000D07FE0444A0025002D00D07CE01678B6
:10820000277963791B023B439E4206D00135EDB2CC
:10821000B6239B009C466244EEE76378222B31D064
:1082200009D8202B11D0212B03D1002923D00120E4
:1082300061E000205FE0232B05D1002949D002290D
:108240004CD0012057E0002055E0002903D002293E
:1082500008D001204FE0063207232100FFF7E0FCA1
:10826000012048E0294B002B48D0911D2800FDF744
:108270006DFF01203FE0063207232100FFF7D0FC0D
:10828000012038E0002903D0022906D0012032E085
:108290002100FFF7A9FC01202DE0A178E3781B0263
:1082A0000B430120190001400E005C0804401371CB
:1082B0004B425941C9B22C32100000F07DFC144BE6
:1082C000002B1DD022003100280000E000BF01205B
:1082D00011E02100FFF788FC01200CE00D4B002B82
:1082E00010D0A378E17809021943280000E000BF0C
:1082F000012000E00020F8BD0020FCE70120FAE7A3
:108300000120F8E70120F6E7688102204D610010A6
:108310000000000000000000F0B5D64600B582B0B5
:1083200001900F0000930024002C0DD0002C19D1D7
:10833000EB78BB421ED0AB78BB4255D00124200065
:1083400002B080BCBA46F0BDB625AD0065433D4BDA
:10835000ED18EB78BB42E9D0AB78BB42E6D00134F4
:10836000E4B2E1E7B022FF3237493848FDF73AFE80
:108370000024E4E710239A46AA4496239B00E918B8
:108380006B461A88504600F0ECFB314B002B1BD09B
:108390006B79FF2B18D0002600E00136009B9E422F
:1083A00012D26A79AB19962189008C4663441B78F6
:1083B0009A42F2D1504600F060FB0028EDD1697975
:1083C000200000E000BFE8E7224B002B04D050461D
:1083D00000F053FB002803D02800FFF711FDAAE7A7
:1083E000200000E000BFF7E71B4B002B02D020006D
:1083F00000E000BF2000FFF769FD002801D0012444
:108400009DE728002C3000F025FB002815D1009BAB
:10841000002B14D09B0601D0012490E7A978019885
:10842000FEF7C6FF041E01D1012488E7A9780023C6
:1084300000220198FFF736F881E701247FE7012445
:108440007DE7C04668810220A0A9001024A8001082
:1084500000000000000000000000000010B5002037
:10846000FEF77AFD041E01D0200010BD292202492A
:108470000248FDF7B7FDF7E7E8A9001024A80010AF
:1084800010B5FEF763FD002800D0012010BD0000EC
:1084900010B502794479072323401B021A43C3789D
:1084A0009B079B0F022B16D0032B2ED0012B01D044
:1084B000002010BD022904D01C4B934204D301209C
:1084C000F7E78023DB00F8E7502219491948FDF748
:1084D00089FD0020EDE7022903D0402A0ED80120B3
:1084E000E7E780239B009A4201D10120E1E758226F
:1084F0000F491048FDF776FD0020DAE75C220C49B1
:108500000C48FDF76FFD0020D3E7022904D040237B
:10851000934204D30120CCE78023DB00F8E76322F9
:1085200003490448FDF75EFD0020C2E7FF03000099
:10853000D4A9001024A8001070B5002503E00E781F
:10854000AD19ADB2891995420AD24C78052CF6D1F5
:108550008E787A34344064000419F609A355EEE7A6
:1085600070BD03008A1890B2884202D39A89904263
:1085700002D95A89801880B2704710B503008A4228
:1085800004D8881A80B29C89A04204D9891A89B279
:108590005889081A80B210BD838801E0C91A89B2CF
:1085A0008B42FBD908007047F0B583B006000191FB
:1085B00011001F00D41AA4B29A4202D24389E41ACD
:1085C000A4B2B588A54205D22A003000FFF7D5FF36
:1085D00030822C00002C02D1002003B0F0BD390005
:1085E0003000FFF7D9FF3168F2885043091801982D
:1085F000FDF766FB0120F0E7F0B583B006009308B5
:108600000CE00B784D782D021D438C782404254313
:10861000CB781B062B43336004313B005F1EBFB297
:10862000002BEED10333100018401A4201D103B0E1
:10863000F0BD00230193020001A8FDF741FB019B5F
:108640003360F4E7F0B5DE4657464E464546E0B5A2
:1086500083B005008A460CA909788488E01A80B2A4
:108660001C1B1419A4B2EE8807007743BFB27443F1
:10867000A4B2A34673432C68A0469844002908D0AE
:1086800001291AD003B0F0BCBB46B246A946A046A9
:10869000F0BD904205D3724341465046FDF710FBB2
:1086A000F0E73A0041465046FDF70AFB29683800DA
:1086B00050445A46FDF704FBE4E7904206D3724368
:1086C00092B241465046FFF797FFDBE703233A009B
:1086D0009A43914641465046FFF78EFF43464B442E
:1086E00003213A000A400F4230D00421891A89B28E
:1086F000081C594500D95846C7B2FF2101405846C9
:10870000441AA1B28B460021019101A804E01A7815
:10871000027001300A000133511EC9B2002AF6D19D
:10872000296804E00A78027001301F0001317B1EC5
:10873000DBB2002FF6D15346019A1A605B46002B3C
:10874000A0D05A465046FFF757FF9BE72968F5E748
:10875000F0B585B00500029103920AAA11880BAA10
:1087600017785C1AA4B28B4202D24289A41AA4B22E
:10877000AE88A64208D2320019002800FFF7FDFE9D
:108780002882298A89B23400002C0DD0039B9C4298
:1087900000D31C002800FFF7FFFE03000097220013
:1087A00002992800FFF74EFF200005B0F0BDF0B59C
:1087B00083B004000D0016001F008069002803D05C
:1087C0000121494200F0F4FCE3899BB2228A01971F
:1087D0000092320029002000FFF7BAFF0500218A2D
:1087E00089B202002000FFF7BCFE2082A0690028A9
:1087F00001D000F0BDFC280003B0F0BD70B582B020
:108800001600950809E00B6803701D0A45701D0CE1
:1088100085701B0EC370043025006C1EA4B2002DA1
:10882000F1D1032332001A401E4201D102B070BDC3
:108830000B68019301A9FDF743FAF7E7F0B5DE46AF
:1088400057464E464546E0B583B005008A460CA91A
:108850000878AC88E11A89B21C1B1419A4B2EE88FE
:108860000F007743BFB27443A4B2A34673432C688E
:10887000A0469844002808D001281AD003B0F0BCC4
:10888000BB46B246A946A046F0BD914205D372430D
:1088900051464046FDF714FAF0E73A00514640468B
:1088A000FDF70EFA2868390051445A46FDF708FAD8
:1088B000E4E7914206D3724392B251464046FFF735
:1088C0009DFFDBE703233A009A4391465146404619
:1088D000FFF794FF43464B4403213A000A400F42FE
:1088E0002ED00421891A89B2081C594500D958464E
:1088F000C7B2FF2101405846441AA1B28B465146E7
:108900000968019101A904E00A781A700131020096
:108910000133501EC0B2002AF6D1286804E00A785C
:10892000027001311F0001307B1EDBB2002FF6D137
:108930005B46002BA2D05A465146FFF75FFF9DE7EA
:108940002868F5E7F0B5CE4600B584B00400894646
:10895000151E039343D04069002803D001214942EA
:1089600000F026FCE789BFB2238A9BB2227A002A54
:108970002AD1A288F91A89B29F4202D26389C91A00
:1089800089B2531A9BB22E1C9D4200D91E1CB6B24E
:1089900039002000FFF700FE0300039A0092320026
:1089A00049462000FFF74AFF320039002000FFF758
:1089B000D8FDE0816069002801D000F0D9FB3000CB
:1089C00004B080BCB946F0BDA688AE4205D8AA1B4B
:1089D000E5885543A9441F00DAE72E00D8E71600C2
:1089E000EDE7F0B583B005000F001400019308AB6C
:1089F0001E7880231B029A4228D84069002803D0A1
:108A00000121494200F0D4FBA869002803D00121CC
:108A1000494200F0CDFB2F60AC80019BEB802E72B1
:108A20006400013CA4B2AC81E4436C810023EB817F
:108A30002B826869002801D000F09AFBA869002801
:108A400006D000F095FB012003B0F0BD0020FBE74D
:108A50000120F9E710B5C3899CB2028A91B29B1A32
:108A60009BB28C4202D242899B1A9BB28288101C14
:108A70009A4200D9181C80B210BD0300C0891B8A1D
:108A8000C01A43425841C0B2704730B5C3899DB245
:108A9000018A8CB282885B1A9BB2A54202D24089BD
:108AA0001B1A9BB2D01A80B230BD70B504000D0005
:108AB0008069002803D00121494200F079FBE28956
:108AC00092B2238A9BB229002000FFF76DFD0500BA
:108AD000218A89B282B22000FFF743FD2082A0697B
:108AE000002801D000F044FB280070BD10B5002321
:108AF000FFF75DFE10BD70B504000D004069002851
:108B000003D00121494200F053FBE3899EB2228A3F
:108B100091B29B1A9BB2B14202D962899B1A9BB255
:108B2000A2889A4202D1207A002817D03100200072
:108B3000FFF732FDE288504323689C4660442900D9
:108B4000FDF7BEF8012231002000FFF70AFDE081A9
:108B50006069002803D000F00BFB012070BD0120EC
:108B6000FCE710B50023FFF7EDFE10BD10B50400C3
:108B70004069002803D00121494200F019FBA06997
:108B8000002803D00121494200F012FB0023E381B9
:108B90002382A3885B00013B9BB2A381DB436381FB
:108BA0006069002801D000F0E3FAA069002801D034
:108BB00000F0DEFA012010BD70B504000D00406920
:108BC000002803D00121494200F0F2FAA0690028F0
:108BD00003D00121494200F0EBFA257260690028B8
:108BE00001D000F0C5FAA069002801D000F0C0FA59
:108BF000012070BD10B5024800F034F810BDC04629
:108C0000488C022010B5002901D000230AE0114B46
:108C1000114A1F311148FBF715F800240DE03732D7
:108C2000C25401334A1E9A420FD90F2B0DD85A084D
:108C30000B4CA25CDC07F0D40424224114000F2268
:108C40002240092AEBDC3032EAE7C0180023037027
:108C500010BDC046F4A9001040AA0010FCA90010E5
:108C6000488C022070B588B0040004AD002604963C
:108C70000922002105A8FDF71DF800960922002110
:108C800001A8FDF717F84B232B700D226946280029
:108C900000F066FA002304E05A1D69468A5CE2543B
:108CA0000133072BF8DD08B070BD000010B50100DE
:108CB0000148F9F7A7FA10BD968E022000B583B0DF
:108CC0000100044B00930B2300220348F9F771FACB
:108CD00003B000BDC8AB0010968E02200523CB5612
:108CE000002B01DB934211D1094B9C466044434267
:108CF00058418000074BC058097901238B40013B44
:108D00009340184043425841C0B270470020FCE7EE
:108D10000000D0AFB885022070B50A79202A19D892
:108D2000174B9C466044434258418000154BC45841
:108D300001239340013B497949B2002910DB080027
:108D40002025AA1A914218DC8B401C4201D0012038
:108D5000404270BD0C4B0D4A40210D48FAF772FF9E
:108D60002020801A002805DB1A0082401442F0D02F
:108D70000138F7E701204042EBE701204042E8E7F5
:108D80000000D0AFB8850220E8AB0010ECAC0010BA
:108D900014AC001070B505000C001600FFF79EFF24
:108DA000002801D0002007E01548FAF7E5FF8319F5
:108DB00012339B005A510130237983420FD9237813
:108DC000617809021943A27812041143E3781B0663
:108DD0000B4342009A5A530BE9D19219E7E701225B
:108DE0009A401300013B074A944665446A42554144
:108DF000B340054AAD00A9580B43AB5070BDC04607
:108E000050AC00100000D0AFB885022010B5054B63
:108E10009C46604443425841800041180248F9F79B
:108E2000F1F910BD0000D0AFA08E022010B582B0C5
:108E30000A4B9C466044434258418400E31C084A64
:108E4000009222000748F9F7B4F9844202DC001BC3
:108E500002B010BD01204042FAE7C0460000D0AF8A
:108E600064AC0010A08E0220F8B505000E00F9F7E2
:108E700071F9070031002800FFF74EFF041E09DBDF
:108E8000020031002800FFF785FF3800F9F76EF97E
:108E90002000F8BD0148FAF76FFFC04650AC001043
:108EA00070B504000B7901259D40013D9540F9F70F
:108EB00051F90C4BE3185A42534199000A4A8A5817
:108EC00029001140A94206D19B00AA4306495A50E5
:108ED000F9F74CF970BD054B054A8A210548FAF7A8
:108EE000B1FEC0460000D0AFB885022088AC0010AB
:108EF000D8AC001014AC001010B50400F9F72AF932
:108F00000A4BE3185A4253419B00094A00219950E9
:108F1000002306E01F2119401A001232920011515D
:108F200001331F2BF6D9F9F721F910BD0000D0AF9E
:108F3000B8850220F0B5CE46474680B581464B0045
:108F40005B18DB004B44DC331B689C460027202465
:108F500017E0AE067B011E434B005B18DB004B4461
:108F6000DC2080469844404606601F261640B046E6
:108F7000E026360240460643D8331E60641B7F1944
:108F80005209002C04D02500052CE2D90525E0E784
:108F90004B005918C90049440800DC30634603609F
:108FA000C0BCB946B046F0BDF0B505AC25784C0064
:108FB0006418E4000419DC342468A446002D01D0B0
:108FC0001F2614E0002612E05401A0256D0525435C
:108FD0004C006418E40004192700DC373D600D4D97
:108FE0003543D8342560053B05321F242240052B2C
:108FF000EAD89B06520113434C006218D200821833
:109000001500DC352B60034B1E43D83216606346D7
:109010002B60F0BD80E00000F0B58BB004000D00C7
:10902000160002680121A9408A430260002B35D056
:1090300069004919C90041180A00C832186810604F
:10904000043258681060043298681060DB68DC31C4
:109050000B6069004B19DB00D033E318802252010A
:109060001343802212061A601A60234BAB40A360A0
:109070002268281D01231F0087403A43226022688E
:10908000280008308340134323601F2216404919EB
:10909000C9006418D83426600BB0F0BD102200213E
:1090A00006A8FCF707FE80235B020693F8235B0209
:1090B00007938023DB020893C0231B03089310222D
:1090C00006A902A8FCF7FCFD6B005B19DB00E318A6
:1090D0001A00C83202991160039A01921A00CC3228
:1090E00001991160049A01921A00D032019911601D
:1090F000059ADC331A60ACE70101010110B5830762
:109100000AD00300032102E001330B4205D01A7894
:10911000002AF9D1181A10BD030019680C4A0D4C29
:109120008A188A4322420FD15968094A04338A189F
:109130008A43224208D15968054A04338A188A436F
:109140002242F1D000E001331A78002AFBD1E1E796
:10915000FFFEFEFE80808080F8B5C0460000000063
:1091600001B40248844601BC604700BF05030020EB
:1091700001B40248844601BC604700BF5102002090
:1091800001B40248844601BC604700BFDD030020F3
:1091900001B40248844601BC604700BFDD030020E3
:1091A00001B40248844601BC604700BF09010020A9
:1091B00001B40248844601BC604700BFDD010020C5
:1091C00001B40248844601BC604700BFC1000020D2
:1091D000636861696E5F746F203C3D204E554D5F42
:1091E000444D415F4348414E4E454C530000000002
:1091F000463A5C5069636F53444B5C5069636F5CE3
:109200007069636F2D73646B5C7372635C72703230
:109210005F636F6D6D6F6E5C6861726477617265BC
:109220005F646D615C696E636C7564652F68617203
:1092300064776172652F646D612E680073697A6569
:10924000203D3D20444D415F53495A455F38207CC5
:109250007C2073697A65203D3D20444D415F534930
:109260005A455F3136207C7C2073697A65203D3D0C
:1092700020444D415F53495A455F3332000000009E
:1092800064726571203C3D20445245515F464F5207
:10929000434500004552525F554E4B4E4F574E5F6F
:1092A0004D53470A000000004C4F4749435F414E71
:1092B000414C595A45525F56335F350A0000000051
:1092C000434150545552455F535441525445440A0A
:1092D00000000000434150545552455F4552524FE3
:1092E000520A000053797374656D20636C6F636B71
:1092F000206F66202575206B487A2063616E6E6F43
:10930000742062652065786163746C79206163689C
:1093100069657665640000002093001009FF000075
:10932000A0802060C7201D40C5001D40450000C032
:10933000080000003C93001008FF0000A08020609F
:109340001D40C4001D40440000C00700549300109D
:1093500008FF0000A08020600040C20000404400E0
:1093600000C007006C93001008FF0000A080206080
:109370000040C4000040440000C007006368616E04
:109380006E656C5F636F6E6669675F7365745F645B
:10939000726571006368616E6E656C5F636F6E66A7
:1093A00069675F7365745F636861696E5F746F009E
:1093B0006368616E6E656C5F636F6E6669675F732D
:1093C00065745F7472616E736665725F6461746107
:1093D0005F73697A65000000020304050607080947
:1093E0000A0B0C0D0E0F101112131415161A1B1C5C
:1093F00068775F69735F636C61696D656428626932
:1094000074732C206269745F696E6465782900004A
:10941000463A5C5069636F53444B5C5069636F5CC0
:109420007069636F2D73646B5C7372635C7270320E
:109430005F636F6D6D6F6E5C68617264776172659A
:109440005F636C61696D5C636C61696D2E630000C4
:1094500068775F636C61696D5F636C656172000062
:109460004E6F207370696E6C6F636B7320617265F1
:1094700020617661696C61626C65000064656C7482
:1094800061203E3D202D3230343820262620646570
:109490006C7461203C3D2032303436202626202159
:1094A0002864656C7461202620312900463A5C509E
:1094B00069636F53444B5C5069636F5C7069636FA1
:1094C0002D73646B5C7372635C7270325F636F6D7B
:1094D0006D6F6E5C68617264776172655F697271ED
:1094E0005C6972712E630000212864656C746120D0
:1094F0003E3E20313175290063757272656E7420AD
:109500003D3D205F5F756E68616E646C65645F757C
:109510007365725F697271207C7C206375727265FD
:109520006E74203D3D2068616E646C6572000000C1
:109530006972715F68616E6465725F636861696EAC
:109540005F667265655F736C6F745F6865616420E8
:109550003E3D203000000000767461626C655F68FB
:10956000616E646C6572203D3D205F5F756E686161
:109570006E646C65645F757365725F69727100001B
:10958000212828282875696E747074725F74297692
:109590007461626C655F68616E646C657229202D10
:1095A00020282875696E747074725F7429697271ED
:1095B0005F68616E646C65725F636861696E5F733A
:1095C0006C6F747329202D2031292573697A656F9A
:1095D0006628737472756374206972715F68616E56
:1095E000646C65725F636861696E5F736C6F742928
:1095F0002900000030783163203D3D20282A696E23
:109600007374293E3E313175000000002165786396
:10961000657074696F6E207C7C20657863657074FA
:10962000696F6E203D3D206E756D202B2031360018
:1096300066616C736500000069735F7368617265D1
:10964000645F6972715F7261775F68616E646C6597
:109650007228736C6F745F68616E646C6572290048
:10966000657863657074696F6E000000666F756E73
:10967000640000004E6F207573657220495251736B
:109680002061726520617661696C61626C650000C1
:109690006972715F6164645F7461696C5F746F5F4C
:1096A000667265655F6C697374000000696E73654E
:1096B00072745F6272616E63685F616E645F6C6931
:1096C0006E6B00006972715F72656D6F76655F68C1
:1096D000616E646C657200006D616B655F627261E2
:1096E0006E6368007265736F6C76655F6272616E3F
:1096F000636800006972715F6164645F73686172BE
:1097000065645F68616E646C657200006972715FA8
:109710007365745F6578636C75736976655F68619E
:109720006E646C657200000072742D3E616C617233
:109730006D5F6964203D3D2069640000463A5C50DD
:1097400069636F53444B5C5069636F5C7069636F0E
:109750002D73646B5C7372635C636F6D6D6F6E5CB5
:109760007069636F5F74696D655C74696D652E63A4
:10977000000000006964202626206964203C3D200A
:10978000706F6F6C2D3E686561702D3E6D61785F06
:109790006E6F646573000000256C6C642028686936
:1097A000202530327829000069642026262069644B
:1097B000203C3D20686561702D3E6D61785F6E6F65
:1097C00064657300463A5C5069636F53444B5C5068
:1097D00069636F5C7069636F2D73646B5C73726334
:1097E0005C636F6D6D6F6E5C7069636F5F757469DC
:1097F0006C5C696E636C7564652F7069636F2F753F
:1098000074696C2F70686561702E68007061726594
:109810006E745F69640000006368696C645F69640A
:1098200000000000706172656E745F696420213D04
:10983000206368696C645F69640000002170685F80
:10984000636F6E7461696E735F6E6F646528706FAD
:109850006F6C2D3E686561702C2072657573655F55
:109860006964290075735F73696E63655F626F6F0A
:1098700074203C3D20494E5436345F4D4158000021
:10988000463A5C5069636F53444B5C5069636F5C4C
:109890007069636F2D73646B5C7372635C636F6D6F
:1098A0006D6F6E5C7069636F5F626173655C696E3A
:1098B000636C7564652F7069636F2F74797065735D
:1098C0002E68000072656D6F7665645F6964203D87
:1098D0003D206E6578745F696400000063616C6CA4
:1098E0006261636B00000000706F6F6C2D3E616CF5
:1098F00061726D5F696E5F70726F677265737320FE
:109900003D3D206D616B655F7075626C69635F6979
:10991000642869645F686967682C206E6578745F85
:10992000696429006964202626202170685F636FBE
:109930006E7461696E735F6E6F64652868656170CF
:109940002C2069642900000064656661756C745F91
:10995000616C61726D5F706F6F6C5F696E69746965
:10996000616C697A6564282900000000616C61728D
:109970006D5F696420213D20706F6F6C2D3E616CBE
:1099800061726D5F696E5F70726F6772657373008D
:1099900072630000417474656D7074656420746F47
:1099A00020736C65657020696E73696465206F66ED
:1099B00020616E20657863657074696F6E206861E0
:1099C0006E646C65723B2075736520627573795F98
:1099D0007761697420696620796F75206D7573747D
:1099E00000000000616C61726D5F706F6F6C5F638F
:1099F000616E63656C5F616C61726D00757064614E
:109A000074655F75735F73696E63655F626F6F74B2
:109A100000000000616C61726D5F706F6F6C5F6160
:109A20006C61726D5F63616C6C6261636B000000FE
:109A30006765745F656E747279000000616C6172B5
:109A40006D5F706F6F6C5F6765745F64656661758D
:109A50006C7400006765745F656E7472795F696429
:109A60005F6869676800000070685F667265655FBF
:109A70006E6F64650000000070685F6164645F631E
:109A800068696C645F6E6F646500000070685F6990
:109A90006E736572745F6E6F6465000070685F67F7
:109AA00065745F6E6F6465006164645F616C6172B0
:109AB0006D5F756E6465725F6C6F636B00000000B4
:109AC000486172647761726520616C61726D2025F6
:109AD0006420616C726561647920636C61696D6595
:109AE0006400000074696D65725F68772D3E696E71
:109AF00074732026203175203C3C20616C61726DAE
:109B00005F6E756D00000000463A5C5069636F53EC
:109B1000444B5C5069636F5C7069636F2D73646B59
:109B20005C7372635C7270325F636F6D6D6F6E5CDD
:109B300068617264776172655F74696D65725C7487
:109B4000696D65722E630000686172647761726589
:109B50005F616C61726D5F7365745F74617267657C
:109B6000740000007570646174655F75735F73697C
:109B70006E63655F626F6F7400000000726F6F74D8
:109B80005F696400463A5C5069636F53444B5C50B4
:109B900069636F5C7069636F2D73646B5C73726370
:109BA0005C636F6D6D6F6E5C7069636F5F75746918
:109BB0006C5C70686561702E630000002170685FE6
:109BC0006765745F6E6F646528686561702C2072CC
:109BD0006F6F745F6964292D3E7369626C696E678B
:109BE000000000002170685F6765745F6E6F6465D8
:109BF00028686561702C20726F6F745F6964292D0D
:109C00003E706172656E74006E65775F7375625F3A
:109C10007472656520213D20686561702D3E726F0C
:109C20006F745F696400000070685F72656D6F76C5
:109C3000655F616E645F667265655F6E6F64650027
:109C400070685F72656D6F76655F616E795F68657C
:109C50006164000070685F6164645F6368696C647C
:109C60005F6E6F646500000070685F6765745F6EAB
:109C70006F646500746F74616C000000463A5C505C
:109C800069636F53444B5C5069636F5C7069636FC9
:109C90002D73646B5C7372635C636F6D6D6F6E5C70
:109CA0007069636F5F73796E635C6D757465782E30
:109CB000630000006D74782D3E636F72652E7370C3
:109CC000696E5F6C6F636B006C6F636B5F69735F72
:109CD0006F776E65725F69645F76616C6964286D29
:109CE00074782D3E6F776E65722900006D74782D43
:109CF0003E656E7465725F636F756E740000000080
:109D00006D757465785F6578697400006D7574654C
:109D1000785F656E7465725F626C6F636B5F756EA2
:109D200074696C007570646174655F75735F7369E5
:109D30006E63655F626F6F74000000002C206675B3
:109D40006E6374696F6E3A20000000006173736582
:109D50007274696F6E2022257322206661696C65BA
:109D6000643A2066696C6520222573222C206C6978
:109D70006E65202564257325730A000031203D3D62
:109D8000202875696E747074725F74296C2D3E732F
:109D900070696E5F6C6F636B00000000463A5C5048
:109DA00069636F53444B5C5069636F5C7069636FA8
:109DB0002D73646B5C7372635C7270325F636F6D82
:109DC0006D6F6E5C7069636F5F72756E74696D65DF
:109DD0005C72756E74696D652E6300000A2A2A2A0A
:109DE0002050414E4943202A2A2A0A000A00000036
:109DF00072756E74696D655F696E6974000000004C
:109E00007372635F66726571203E3D206672657194
:109E100000000000463A5C5069636F53444B5C504D
:109E200069636F5C7069636F2D73646B5C737263DD
:109E30005C7270325F636F6D6D6F6E5C68617264CF
:109E4000776172655F636C6F636B735C636C6F6388
:109E50006B732E6300000000636C6F636B5F636F56
:109E60006E6669677572650076636F5F66726571AD
:109E7000203E3D20285049434F5F504C4C5F564395
:109E80004F5F4D494E5F465245515F4D485A202A1B
:109E9000204D485A292026262076636F5F6672651A
:109EA00071203C3D20285049434F5F504C4C5F5639
:109EB000434F5F4D41585F465245515F4D485A20D0
:109EC0002A204D485A290000463A5C5069636F5376
:109ED000444B5C5069636F5C7069636F2D73646B96
:109EE0005C7372635C7270325F636F6D6D6F6E5C1A
:109EF00068617264776172655F706C6C5C706C6CC9
:109F00002E6300006662646976203E3D2031362073
:109F10002626206662646976203C3D20333230007C
:109F200028706F73745F64697631203E3D20312064
:109F3000262620706F73745F64697631203C3D2063
:109F400037292026262028706F73745F6469763263
:109F5000203E3D203120262620706F73745F646997
:109F60007632203C3D20372900000000706F73746A
:109F70005F64697632203C3D20706F73745F646962
:109F8000763100007265665F6D687A203C3D20285E
:109F900076636F5F66726571202F2031362900006D
:109FA000706C6C5F696E697400000000666E690019
:109FB000666E692B000000006E616E00666E692D92
:109FC00000000000AE4D00105E4D00105E4D001010
:109FD000B84D00105E4D00105E4D00105E4D00103B
:109FE0005E4D00105E4D00105E4D00105E4D001085
:109FF000A44D00105E4D00109A4D00105E4D0010F3
:10A000005E4D0010904D0010504E0010764E001026
:10A010008E4E0010764E0010304E0010764E00101E
:10A02000764E0010764E0010764E0010764E0010E0
:10A03000764E0010764E00106C4E0010764E0010DA
:10A04000764E0010764E0010764E0010764E0010C0
:10A050009A4E0010CA520010E0520010E052001058
:10A06000E0520010E0520010E0520010E0520010E8
:10A07000E0520010E0520010E0520010E0520010D8
:10A08000E0520010E0520010E0520010E0520010C8
:10A09000E0520010E0520010E0520010E0520010B8
:10A0A000E0520010E0520010E0520010E0520010A8
:10A0B000E0520010E0520010E0520010E052001098
:10A0C000E0520010E0520010E0520010E052001088
:10A0D000E0520010F2500010B2500010F250001088
:10A0E000E0520010E0520010E0520010E052001068
:10A0F000E0520010E0520010E0520010E052001058
:10A10000E0520010E0520010E0520010E052001047
:10A11000E0520010E0520010E0520010E052001037
:10A12000A64E0010E0520010E0520010E052001065
:10A13000E0520010E0520010E0520010E052001017
:10A14000E0520010E0520010A64E001042510010E4
:10A15000A64E0010F2500010B2500010F250001045
:10A16000E0520010A64E0010E0520010E052001025
:10A17000E0520010E0520010E0520010A64E001015
:10A1800094520010E0520010E0520010BA5100103A
:10A19000E0520010A64E0010E0520010E0520010F5
:10A1A000A64E001000000000000000000000F03F7C
:10A1B00000000000000024400000000000005940A2
:10A1C0000000000000408F40000000000088C340F5
:10A1D00000000000006AF8400000000080842E416A
:10A1E00000000000D01263410000000084D79741B6
:10A1F0000000000065CDCD416D697373696E672005
:10A20000646F75626C652066756E6374696F6E004D
:10A210002A282875696E74385F74202A292828280E
:10A22000766F6964202A29726F6D5F646174615F63
:10A230006C6F6F6B757028726F6D5F7461626C65A7
:10A240005F636F6465282753272C20274627292919
:10A25000292D322929202A2034203E3D2053465FD3
:10A260005441424C455F56325F53495A4500000005
:10A27000463A5C5069636F53444B5C5069636F5C52
:10A280007069636F2D73646B5C7372635C727032A0
:10A290005F636F6D6D6F6E5C7069636F5F646F7528
:10A2A000626C655C646F75626C655F696E69745F32
:10A2B000726F6D2E630000005F5F61656162695FB0
:10A2C000646F75626C655F696E6974002A28287511
:10A2D000696E74385F74202A2928726F6D5F74610B
:10A2E000626C652D322929202A2034203E3D2053DE
:10A2F000465F5441424C455F56325F53495A4500D0
:10A30000463A5C5069636F53444B5C5069636F5CC1
:10A310007069636F2D73646B5C7372635C7270320F
:10A320005F636F6D6D6F6E5C7069636F5F666C6F9E
:10A3300061745C666C6F61745F696E69745F726F83
:10A340006D2E63005F5F61656162695F666C6F615E
:10A35000745F696E6974000044656275670000008F
:10A36000626F6F74325F77323571303830000000C1
:10A37000332E3000312E342E300000007069636FB0
:10A380005F7700004C6F676963416E616C797A6535
:10A3900072000000466562202034203230323300E3
:10A3A00006005250BBFF3CB67CA300100600525082
:10A3B0003ABCA91170A3001006005250E182887FB8
:10A3C00060A3001006005250D3F0754258A300104D
:10A3D0006C656E203D3D203100000000463A5C5027
:10A3E00069636F53444B5C5069636F5C7069636F62
:10A3F0002D73646B5C7372635C7270325F636F6D3C
:10A400006D6F6E5C7069636F5F737464696F5C73AA
:10A410007464696F2E6300007570646174655F75A4
:10A42000735F73696E63655F626F6F740000000035
:10A43000676574636861725F74696D656F75745F79
:10A44000757300000D0A000085600010896000101F
:10A4500095600010E5600010C96000100000000069
:10A46000737464696F5F7573625F636F72655F6E4B
:10A47000756D203D3D206765745F636F72655F6E2B
:10A48000756D282900000000463A5C5069636F53DF
:10A49000444B5C5069636F5C7069636F2D73646BD0
:10A4A0005C7372635C7270325F636F6D6D6F6E5C54
:10A4B0007069636F5F737464696F5F7573625C73F7
:10A4C0007464696F5F7573622E6300005553422098
:10A4D000737464696E202F207374646F7574000048
:10A4E0000600525053B4F4A1CCA4001075706461FE
:10A4F00074655F75735F73696E63655F626F6F74B8
:10A500000000000074696D65725F7461736B000018
:10A5100052617370626572727920506900000000A8
:10A520005069636F00000000426F61726420434411
:10A530004300000052657365740000000902540076
:10A54000030100807D080B000202020000090400E4
:10A55000000102020004052400200105240100017D
:10A5600004240202052406000107058103080010E7
:10A5700009040100020A0000000705020240000071
:10A58000070582024000000904020000FF000105E7
:10A5900012010002EF0201408A2E0A0000010102AE
:10A5A000030100000000000010A5001020A500100D
:10A5B000808E022028A5001034A500102828756977
:10A5C0006E747074725F7420296E6578745F627542
:10A5D000666665725F707472202620306231313198
:10A5E0003131317529203D3D20300000463A5C5024
:10A5F00069636F53444B5C5069636F5C7069636F50
:10A600002D73646B5C6C69625C74696E79757362DE
:10A610005C7372635C706F727461626C655C7261B2
:10A620007370626572727970695C72703230343046
:10A630005C6463645F7270323034302E63000000FB
:10A6400068775F646174615F6F6666736574286EB6
:10A650006578745F6275666665725F7074722920D2
:10A660003C3D205553425F445052414D5F4D41584F
:10A6700000000000556E68616E646C65642049528C
:10A680005120307825780A007268706F7274203D0E
:10A690003D2030006463645F656470745F78666554
:10A6A000720000006463645F656470745F6F70655E
:10A6B0006E0000006463645F7365745F616464725C
:10A6C000657373006463645F696E745F656E616275
:10A6D0006C6500005F68775F656E64706F696E74AB
:10A6E0005F616C6C6F6300006463645F696E6974C2
:10A6F0000000000021286275665F6374726C20267A
:10A70000205553425F4255465F4354524C5F465575
:10A710004C4C2900463A5C5069636F53444B5C5083
:10A7200069636F5C7069636F2D73646B5C6C6962E5
:10A730005C74696E797573625C7372635C706F725E
:10A740007461626C655C726173706265727279705B
:10A75000695C7270323034305C7270323034305F29
:10A760007573622E630000006275665F6374726CBD
:10A770002026205553425F4255465F4354524C5F5A
:10A7800046554C4C00000000657020256420257360
:10A790002077617320616C726561647920617661F4
:10A7A000696C61626C6500005741524E3A207374C7
:10A7B000617274696E67206E6577207472616E7362
:10A7C000666572206F6E20616C72656164792061CC
:10A7D00063746976652065702025642025730A00FE
:10A7E00043616E277420636F6E74696E756520789F
:10A7F000666572206F6E20696E616374697665208C
:10A800006570202564202573000000006F757400BA
:10A81000696E000073796E635F65705F627566666E
:10A820006572000025732025643A20415353455238
:10A8300054204641494C45440D0A0000F86E001072
:10A84000566E0010866E0010C26E0010F86E00107A
:10A85000F86E0010DE6E0010866E0010F86E0010AC
:10A86000F86E0010F86E0010F86E0010F86E001010
:10A87000F86E0010F86E0010686E00107A77001005
:10A8800054770010307900102E77001030790010C6
:10A89000967600102277001030790010B276001002
:10A8A000CA7600109679001088790010DA790010C5
:10A8B0004A7B0010C67A0010E67A0010EE7900108C
:10A8C0003A7A00104E7B0010757362645F656470A5
:10A8D000745F786665720000757362645F656470AA
:10A8E000745F6F70656E0000757362645F6F706592
:10A8F0006E5F656470745F70616972006F73616C24
:10A900005F71756575655F73656E640070726F6306
:10A910006573735F6765745F646573637269707490
:10A920006F72000070726F636573735F7365745F3D
:10A93000636F6E666967000070726F636573735F43
:10A94000636F6E74726F6C5F72657175657374009E
:10A950007475645F7461736B00000000ED7F00101C
:10A96000A9800010ED800010E5810010198300100F
:10A9700000000000757362645F636F6E74726F6CC9
:10A980005F786665725F6362000000007475645FE3
:10A99000636F6E74726F6C5F7866657200000000A2
:10A9A000636463645F786665725F636200000000E1
:10A9B000636463645F6F70656E0000007475645F4C
:10A9C0006364635F6E5F77726974655F666C7573ED
:10A9D0006800000074755F656470745F76616C690F
:10A9E0006461746500000000747573625F696E696C
:10A9F000740000006C656E203E203000463A5C50CA
:10AA000069636F53444B5C5069636F5C7069636F3B
:10AA10002D73646B5C7372635C7270325F636F6D15
:10AA20006D6F6E5C7069636F5F756E697175655F80
:10AA300069645C756E697175655F69642E63000099
:10AA40007069636F5F6765745F756E697175655F67
:10AA5000626F6172645F69645F737472696E6700CC
:10AA6000666C6173685F6F666673202B20636F7519
:10AA70006E74203C3D205049434F5F464C41534843
:10AA80005F53495A455F425954455300463A5C501A
:10AA900069636F53444B5C5069636F5C7069636FAB
:10AAA0002D73646B5C7372635C7270325F636F6D85
:10AAB0006D6F6E5C68617264776172655F666C6110
:10AAC00073685C666C6173682E630000636F6E6E02
:10AAD0006563745F696E7465726E616C5F666C61EC
:10AAE000736820262620666C6173685F65786974D8
:10AAF0005F78697020262620666C6173685F7261DA
:10AB00006E67655F657261736520262620666C61DD
:10AB100073685F666C7573685F6361636865000086
:10AB2000636F6E6E6563745F696E7465726E616C7F
:10AB30005F666C61736820262620666C6173685FAF
:10AB4000657869745F78697020262620666C617369
:10AB5000685F72616E67655F70726F6772616D20AA
:10AB6000262620666C6173685F666C7573685F6328
:10AB70006163686500000000636F6E6E6563745FFB
:10AB8000696E7465726E616C5F666C6173682026B5
:10AB90002620666C6173685F657869745F78697098
:10ABA00020262620666C6173685F666C7573685F2B
:10ABB0006361636865000000666C6173685F646F61
:10ABC0005F636D64000000004E6F20444D412063C0
:10ABD00068616E6E656C7320617265206176616973
:10ABE0006C61626C6500000070726F6772616D2D40
:10ABF0003E6C656E677468203C3D2050494F5F494C
:10AC00004E535452554354494F4E5F434F554E5443
:10AC100000000000463A5C5069636F53444B5C503F
:10AC200069636F5C7069636F2D73646B5C737263CF
:10AC30005C7270325F636F6D6D6F6E5C68617264C1
:10AC4000776172655F70696F5C70696F2E63000079
:10AC50004E6F2070726F6772616D207370616365F3
:10AC6000000000004E6F2050494F207374617465DE
:10AC7000206D616368696E6573206172652061761D
:10AC800061696C61626C650070726F6772616D5FA3
:10AC90006D61736B203D3D20285F757365645F694E
:10ACA0006E737472756374696F6E5F7370616365E0
:10ACB0005B70696F5F6765745F696E646578287043
:10ACC000696F295D20262070726F6772616D5F6DFC
:10ACD00061736B290000000070696F5F72656D6FB2
:10ACE00076655F70726F6772616D00005F70696F8B
:10ACF0005F66696E645F6F66667365745F666F72C8
:0CAD00005F70726F6772616D00000000F0
:10AD0C00B4020010A80200109C020010A0A30010B6
:10AD1C0090020010ACA30010B8A30010C4A3001044
:04AD2C00E0A400108F
:10AD300010B5D0231B0600241C570268EFF31081C6
:10AD400072B61368002BFCD0BFF35F8F0423C35689
:10AD5000002B08DB0368BFF35F8F00221A6081F3CA
:10AD6000108820BFE9E704710368BFF35F8F0022FA
:10AD70001A6081F3108810BD03000068EFF3108C97
:10AD800072B60268002AFCD0BFF35F8F04229A5685
:10AD9000002A0BDB002910D00A6000201B68BFF3DB
:10ADA0005F8F00221A608CF310887047D022120641
:10ADB000127852B21A710120F0E70020EEE700008D
:10ADC000F8B5CE46474680B504001700984603689C
:10ADD000002B20D0D0231B061B785BB29946266837
:10ADE000EFF3108C72B63568002DFCD0BFF35F8F87
:10ADF00004256557002D14DB2368BFF35F8F002205
:10AE00001A608CF310883800414600F031F90028B0
:10AE1000E5D000200FE00A4B0A4A7A210A4800F0E8
:10AE200017F94B4623712368BFF35F8F00221A6026
:10AE30008CF310880120C0BCB946B046F8BDC046AE
:10AE4000B49C00100C9D00107C9C0010F0B5C64610
:10AE500000B582B00700884600F002F904000D1E1C
:10AE60001CDB0190FA22920000234046002100F0F2
:10AE700007F922002B0012184B419D4202D804D141
:10AE8000944202D901225242D317002B0CDB380026
:10AE9000FFF796FF02B080BCB846F0BD054B064AEE
:10AEA0003F21064800F0D4F8024B034A3F210348F3
:10AEB00000F0CEF864980010249D001080980010D7
:10AEC00010B50268EFF3108172B61368002BFCD046
:10AED000BFF35F8F0423C356002B0ADBFF230371EC
:10AEE0000368BFF35F8F00221A6081F3108840BFB0
:10AEF00010BD034B034AA921034800F0A9F8C0463E
:10AF0000C89C0010009D00107C9C0010094B1B7811
:10AF1000002B08D00CE09A008021490551180868E0
:10AF20000549505001333F2BF5DD024B01221A70C9
:10AF30007047C0469A8E0220D085022010B5024B81
:10AF40000133984710BDC046D085022000280AD0A2
:10AF500003231B02054A12685340C022920013408B
:10AF6000034A136070470223F3E7C0460C80014098
:10AF70000C900140F0B5D6464F464646C0B5070096
:10AF80000E00150018239A461B881422904610883C
:10AF900028499847814653461B88424610882649CF
:10AFA0009847040053461B88424610882349984717
:10AFB00080464B46002B0CD0002C0AD0002808D02D
:10AFC000FFF7A4FFC847A0470020FFF7BFFF2A00F4
:10AFD0000FE01B4B1B4A80211B4800F039F8002B67
:10AFE00007D0002A05D0C0235B051B6E3370013AE1
:10AFF00001362B00134312D0C0235B059C6A082343
:10B000002340A107EBD5002DE9D0511B0D29E6D82F
:10B010003878C02149050866013D0137DFE7012086
:10B02000FFF794FFC047FFF789FFE0BCBA46B1467F
:10B03000A846F0BD494600004558000046430000C0
:10B0400078AB0010B8AB00108CAA00107047C04657
:10B0500001B40248844601BC604700BF453C001073
:10B0600001B40248844601BC604700BF253500108A
:10B0700001B40248844601BC604700BF013400109F
:10B0800001B40248844601BC604700BF395B001030
:10B090002804002009FF0000A080206000E007C015
:10B0A000E0A04460A40001E0080000002481022028
:10B0B000200010000000000000000100000000005F
:10B0C000000000000000020000000000000000007E
:10B0D0000000030000000000000000000000FF006E
:10B0E0000000000000B5486801318E4600477046F8
:10B0F00009380149884700BD1D280010A40400201C
:10B1000000000000008002200487022000000000F0
:10B110000000000014870220000000000000000072
:10B12000100000000000000000000000000000000F
:10B13000503300004C330000543300005233000001
:10B140004D5300004D4300005334000043340000D1
:10B150000562001000000000756100100000000092
:10B16000000100000CA8001010A80010F8840220B4
:10B1700010000C000000E0FF1F00000000000000B5
:10B1800000000000000000000000000000000000BF
:10B1900000000000000000000000000000000000AF
:10B1A000A55C001045530010395A00101D5C0010BA
:08B1B000ED020010F58B001008
:04000005100001E9FD
:00000001FF
